:020000040800F2
:10000000C8190020B90200089D36000861330008B5
:100010006B360008B51C00088D6200080000000067
:10002000000000000000000000000000DD420008A9
:10003000D127000800000000ED37000851490008F2
:10004000D3020008D3020008D3020008D30200083C
:10005000D3020008D3020008D3020008D30200082C
:10006000D3020008D3020008D3020008D30200081C
:10007000D3020008D3020008D3020008D30200080C
:10008000D3020008D3020008D3020008D3020008FC
:10009000D3020008D3020008D30200087529000823
:1000A000D3020008D3020008D3020008D3020008DC
:1000B000D3020008D3020008D3020008D3020008CC
:1000C000D3020008D3020008D3020008D3020008BC
:1000D000D3020008615C0008D3020008D3020008C4
:1000E000D3020008D3020008D3020008D30200089C
:1000F000D3020008D3020008D3020008D30200088C
:10010000D3020008D3020008D3020008D30200087B
:10011000D3020008D3020008D3020008D30200086B
:10012000D3020008D3020008D3020008D30200085B
:1001300000F002F800F0B0F80AA090E8000C824449
:100140008344AAF10107DA4501D100F0A5F8AFF226
:10015000090EBAE80F0013F0010F18BFFB1A43F0A5
:1001600001031847B0690000D06900000A444FF04D
:10017000000C10F8013B13F0070408BF10F8014B06
:100180001D1108BF10F8015B641E05D010F8016B4B
:10019000641E01F8016BF9D113F0080F1EBF10F8AF
:1001A000014BAD1C0C1B09D16D1E58BF01F801CBD2
:1001B000FAD505E014F8016B01F8016B6D1EF9D555
:1001C0009142D6D37047000000230024002500266A
:1001D000103A28BF78C1FBD8520728BF30C148BFAA
:1001E0000B6070476E2900F0E981702900F02B83C5
:1001F000662906F0B583652906F0B283672906F003
:10020000AF836129AFF3008003681B0A28BF41F068
:100210008001692900F09681642900F09381752995
:1002200000F090816F2900F0B882782900F0F78201
:10023000E92900F05382E42900F05082F52900F00A
:100240004D82EF2900F0B582F82900F0F6820368AC
:10025000DB0928BF41F08001632900F0AC867329D7
:1002600000F0B186E32900F0BC86F32900F0C186D6
:10027000002070471FB500F00DFF04000020002192
:1002800006F058FB401C60600020002106F03CFB9B
:10029000E0601FBD10B510BD00F0CFFE1146FFF7A6
:1002A000E9FF06F00FFA00F0ABFF03B4FFF7F2FF2F
:1002B00003BC00F0F3FF00000948804709480047ED
:1002C000FEE7FEE7FEE7FEE7FEE7FEE7FEE7FEE706
:1002D000FEE7FEE704480549054A064B7047000063
:1002E0008149000831010008C8130020C819002006
:1002F000C8150020C81500201CB50C46064B7B44D1
:1003000069460090204600F072F9044600206946D4
:1003100000F080F920461CBD1303000040EA0103F1
:10032000024630B59B0710D14FF0013400E008C2FF
:1003300008C91D1B9D4315EAC41FF8D013F0FF0127
:1003400002F8011B0DD01B0AF8E711F8013B002B46
:1003500002F8013B05D011F8013B002B02F8013BEC
:10036000F3D130BD10B5431C02E010F8011B71B190
:100370008107FAD14FF0013202C88C1A8C4314EA7B
:10038000C211F9D0C01A0A0603D0C01E10BDC01A8F
:1003900010BD0A0401D0801E10BD0902FCD0401E11
:1003A00010BD032A40F2308010F0030C00F01580DD
:1003B00011F8013BBCF1020F624498BF11F801CB68
:1003C00000F8013B38BF11F8013BA2F1040298BFCD
:1003D00000F801CB38BF00F8013B11F0030300F037
:1003E0000183083AC0F0088051F8043B083A51F8FC
:1003F00004CBA0E80810F5E7121D5CBF51F8043BE0
:1004000040F8043BAFF30080D20724BF11F8013B52
:1004100011F801CB48BF11F8012B24BF00F8013BB4
:1004200000F801CB48BF00F8012B70474FF00002E5
:1004300000B5134694469646203922BFA0E80C50DA
:10044000A0E80C50B1F12001BFF4F7AF090728BFB5
:10045000A0E80C5048BF0CC05DF804EB890028BF31
:1004600040F8042B08BF704748BF20F8022B11F05A
:10047000804F18BF00F8012B7047704770477047D6
:1004800070B5044685690068C10601D5302600E0D4
:100490002026C00707D070BDD4E90121304690471F
:1004A000206A401C20626D1EF6D570BD70B50446F2
:1004B00085690078C00707D170BDD4E901212020EB
:1004C0009047206A401C20626D1EF6D570BD0968F9
:1004D0004A0501D540B27047C905FCD500B2704746
:1004E00009684A0501D5C0B27047C905FCD580B27C
:1004F000704770B50C460546012A05D0287880065D
:1005000000D5EA69002302E0012305E05B1C934269
:1005100002D2E05C0028F9D1A869E618C01AA861E7
:10052000286A184428622846FFF7AAFF04E0D5E9A4
:10053000012114F8010B9047B442F8D32846FFF785
:10054000B5FF70BD2DE9F0410646002410687529FD
:10055000314616A510D0FFF7BAFF002802DA404254
:1005600013A507E031688A0701D512A502E0490703
:1005700004D511A5012401E0FFF7B2FF00210A22F2
:1005800006F1240709E0B0FBF2FCB0FBF2F302FB3A
:100590001C00303078541846491C0028F3D12346FB
:1005A0002A463046BDE8F04100F093BA0000000052
:1005B0002D0000002B0000002000000011680268E0
:1005C000006A530501D508700AE0D30501D50880FB
:1005D00006E0130603D5C217C1E9000200E0086077
:1005E0000120704701694A1C02610878704700B514
:1005F0008FB0CDE901310021059105497944CDE95C
:1006000003101146684600F029F90FB000BD000044
:10061000E5FFFFFF0A6802F8010B0A60704700005F
:100620002DE9FF5F15468A460446DFF8AC80F844A2
:100630000027D8E900103E46CDE9001010E03AF856
:1006400016106A4602A800F0D8FC411C07D0217899
:10065000890603D5E269391891420DD80744761C02
:100660002078800602D5E069B84205DDAE42E6DBBF
:100670003AF816000028E2D1A069C01BA06120460C
:10068000FFF7FEFED8E90010CDE90010002017E0CA
:100690003AF818106A4602A800F0AFFCB0F1FF3F2C
:1006A00081460BD000250DF1080B05E0D4E90121AE
:1006B0001BF8050090476D1C4D45F7D308F101006C
:1006C000B0428046E4DB206A384420622046FFF7CF
:1006D000EDFEBDE8FF9F0000C66300002DE9F0417C
:1006E0008046D21D22F007020025D2E90002F5293A
:1006F00015A614D0011E72F1000106DA0023D0EB1A
:10070000030063EB020211A608E0D8F800108B0783
:1007100001D50FA602E0490701D50EA60125114615
:10072000002408F1240704E000F08EF930323A5535
:10073000641C50EA0102F7D12B463246214640465E
:10074000BDE8F04100F0C5B9000000002D00000038
:100750002B0000002000000030B4002100F1240430
:1007600008E002F00705D208303542EA4372DB08A0
:100770006554491C52EA0305F3D10468002310A212
:10078000250707D5A40600D421B1C46901230DA211
:10079000641EC46130BC00F09CB910B5044621460B
:1007A0001068FFF79DFE02462046BDE8104000237A
:1007B000D2E7D21D22F00701D1E90023CCE70000E7
:1007C0000000000030000000F0B40D46018809056B
:1007D00002D5214C7C4402E01F4C7C440E340021A5
:1007E00000F1240608E002F00F071209E75D42EA73
:1007F00003721B097754491C52EA0307F3D10278AC
:100800000023120704D5702D06D009B1022311343C
:100810002246F0BC00F05DB901231034F8E770B552
:1008200004460D4621461068FFF75AFE0246294647
:100830002046BDE870400023C6E7D21D22F0070322
:10084000D3E90023C0E70368126843F02003036084
:100850000823C3610023B7E7286200002DE9F05F99
:10086000894604464FF0000ADFF874B1FB44C0F833
:1008700020A02046E1688847002874D0252806D0AB
:10088000D4E901219047206A401C2062F1E700264C
:100890005F462046E16888472028054607DB312D62
:1008A00005D2781910F8200C08B10643F1E7B0071B
:1008B00001D526F00406C4F81CA00027C4F818A02F
:1008C0002A2D09D0284605F0E0FE38B304EB87084E
:1008D000303DC8F8185019E059F8041B204604EBC5
:1008E00087029161E1688847012F054618D1E069C8
:1008F000002820DA26F020061DE0D8F8180000EBCA
:10090000800005EB40003038C8F818002046E16848
:100910008847054605F0B9FE0028EED1012F0AD020
:100920002E2D08D12046E16888477F1C0546022FFE
:1009300046F02006C4DBA069002803DA404246F0F6
:100940000106A061F00701D026F010066C2D0BD037
:10095000682D09D04C2D39D06A2D35D0742D35D065
:100960007A2D33D016E038E0E1682F4620468847DC
:10097000B842054609D16C2F26D04FF48060E1685B
:10098000064320468847054604E06C2F1AD04FF4F2
:10099000807006430DB3A5F14100192802D8203517
:1009A00046F400664A462946204626604E46FFF732
:1009B00019FC80B101280BD0F61D26F0070000F1CC
:1009C000080956E74020E4E78020D8E70020D6E772
:1009D00006F104094DE7284652E7206ABDE8F09F7A
:1009E000B861000010B5203AC0F00B80B1E8185093
:1009F000203AA0E81850B1E81850A0E81850BFF409
:100A0000F5AF5FEA027C24BFB1E81850A0E81850A7
:100A100044BF18C918C0BDE810405FEA827C24BFFB
:100A200051F8043B40F8043B08BF7047D20728BF89
:100A300031F8023B48BF11F8012B28BF20F8023BD8
:100A400048BF00F8012B704730B5B0F10A024FEAF9
:100A5000900E71F100034EEA817EB0EB0E0061EB67
:100A600091014FEA101E4EEA017E10EB0E0041EBA1
:100A700011114FEA102E4EEA016E10EB0E0041EB01
:100A800011214FEA104E4EEA014E10EB0E0041EBE1
:100A90001141401841F100014FEAD00040EA417095
:100AA0004FEAD10110EB80054FEA810444EA9074CB
:100AB00044EB01046D1944EB0404521BA3414FF0B5
:100AC000000348BF0A3200D530BD401C41F100018F
:100AD00030BD2DE9F0470D4699469246044600F197
:100AE00024080168880604D5E06921F0100121601E
:100AF00000E00120A84201DD471B00E00027A169BA
:100B00007A1902EB0900081AA0612078C00602D405
:100B10002046FFF7B5FC002608E0D4E901211AF8C9
:100B200006009047206A401C761C20624E45F4DB8C
:100B30002078C0060AD52046FFF7A2FC06E0D4E9DB
:100B4000012130209047206A401C2062381EA7F106
:100B50000107F4DC07E0D4E9012118F8050090470B
:100B6000206A401C2062281EA5F10105F3DC204606
:100B7000FFF79CFC2078000602D50220BDE8F08734
:100B80000120FBE770472DE9FF4F0C461E464FF052
:100B9000FF378BB0D2E90001DDF860800A908A4609
:100BA000C1F30A5505B93D46002108464FF0000043
:100BB000BAF1000F00F4400005DA00EB80004FF4BA
:100BC000400101EA50004FEA9059B9F1010F00DDF0
:100BD000B9460A9850EA4A000ED044F61050A5F2E1
:100BE000FF3545432F14B8F1000F1ED07542291E62
:100BF0001EDDC9F100021CE0B8F1010F4FF000004A
:100C000001D0302103E0F24305E02154401CB04202
:100C1000FBDB30460022002121540B99C1F80880EB
:100C2000C1E900200FB0BDE8F08FBD1B6D1CDEE7F1
:100C30004A4600DA694206A800F070FA06AB93E86B
:100C4000070003AB83E8070050460A9900F02DFB2C
:100C50008DE80700A0F500501F3800900398002D84
:100C60000ADD42F21F014A460844002303A903900B
:100C7000684600F096FD09E0A0F500504A461F388E
:100C8000002303A90390684600F0A0FD8DE807004B
:100C90000004000C03D04FF0FF30410800E0104684
:100CA000B8F1000F03D00022009215461EE0751E19
:100CB00005D4FFF7C9FE303262556D1EF9D5B34633
:100CC0000122084302D000227F1C04E02078302853
:100CD00001D100227F1E002A099784D01DE0112D2A
:100CE00007DAFFF7B1FE303262556D1C50EA01029F
:100CF000F5D1084302D00098C8B10EE00021681E6B
:100D000005E0235C625C63542254401E491C81420E
:100D1000F7DBAB46A81B401E0990002004F80B002F
:100D20000B98099AC0F80880C0E9002B7AE71126D1
:100D30004FF0000857E72DE9F04F88460446D21DD2
:100D400022F0070191B0D1E90001CDE90A0105F0D7
:100D500088FC02460B98C00F01D02D2007E02068C8
:100D6000810701D52B2002E0202101EAC000032ADF
:100D7000099001D0072A05DB03464146204600F0D2
:100D80008DF90BE12078800601D5E06900E00620AE
:100D9000B8F1650F814606D0B8F1660F18D0B8F1EA
:100DA000670F70D131E00020B9F1110F009001DB25
:100DB000112301E009F101030AAA01A90CA8FFF718
:100DC000E2FEDDE90C70002609F10105834647E0EB
:100DD00001204B4600904FF000470AAA01A90CA839
:100DE000FFF7D1FEDDE90DB00C995D46002610B984
:100DF00009F101000D18B9EB050003D4C0F1FF366D
:100E000009F10105A5EB09002BE0B9F1010F01DAA9
:100E10004FF001090020B9F1110F0090484601DDA3
:100E2000112300E003460AAA01A90CA8FFF7ABFEB4
:100E3000DDE90C704D4600268346207800070AD471
:100E4000AB4500DA5D4601A8012D04DD411911F81A
:100E5000011C302907D04F4502DA17F1040F04DADC
:100E6000012082460FE06D1EEEE7002F02DCED1B35
:100E70003E4403E0781CA84200DD7D1CB81B00F155
:100E8000010A4FF000472078000703D4AA4501DB90
:100E90004FF0FF3A0021B7F1004F0DF143088DF8F4
:100EA000431024D002202B23002F01DA7F422D2370
:100EB0000A21021EA0F1010000DC5FB197FBF1FCEA
:100EC00097FBF1F201FB1C7C17460CF1300C08F883
:100ED00001CDEEE7A8F1010003702188090501D5D5
:100EE000452100E06521A0F1010800F8011C0998E6
:100EF0000FA9A1EB0807FF1D00B10120411901EB6B
:100F0000EA70A1693844081A401EA0612078C00622
:100F100002D42046FFF7B4FA099828B1D4E9012198
:100F20009047206A401C20622078C00622D52046C7
:100F3000FFF7A6FA1EE0002E04DBB34502DD01A890
:100F4000805D00E03020D4E901219047206A401CF8
:100F50002062761CAAF101005FEA000A0AD100F0C3
:100F600099F8C0680168405CD4E901219047206A83
:100F7000401C2062281EA5F10105DCDC07E0D4E955
:100F8000012118F8010B9047206A401C2062381E8E
:100F9000A7F10107F3DC2046FFF788FA032011B020
:100FA00041E610B5436913B1AFF3008001E0FFF7EC
:100FB000A0FA012010BD127800F124010A7000226D
:100FC0004A700122EDE711684FF0FF32E9E710B5F2
:100FD000436913B1AFF3008001E0FFF721FB01206B
:100FE00010BD128800F1240182840022C2840122F3
:100FF000EDE711684FF0FF32E9E770B516460C4691
:10100000054600F03FF8036893F80101012806D077
:10101000FF2C0FD8185D68B101202C7070BDD3F87B
:1010200007013246214603F2071303442846BDE870
:10103000704018474FF0FF3070BD754600F0EAF879
:10104000AE4605006946534620F00700854618B0B5
:1010500020B5FFF73FF9BDE820404FF000064FF004
:1010600000074FF000084FF0000B21F00701AC46DD
:10107000ACE8C009ACE8C009ACE8C009ACE8C009FC
:101080008D46704710B500F005F8001D10BD00BF7B
:10109000A558000000487047841300202DE9F04156
:1010A0001F46044603260168072A01F4006004DB9A
:1010B00008B116A505E016A503E008B115A500E0E6
:1010C00015A521F010002060A069C01EA0610FB11D
:1010D000401EA0612046FFF7D3F94FB1D4E90121AA
:1010E00038469047206A401C2062C01C206206E0FF
:1010F000206AFAE7D4E9012115F8010B9047761E22
:10110000F8D22046FFF7D2F9BDE8F0814E414E00FB
:101110006E616E00494E4600696E66002DE9F0472B
:10112000814616468AB0354878440DC88DE80D00D2
:1011300032487844801C03AC0DC884E80D0041F6A9
:101140009B300844372190FBF1F290FBF1F5A5F1BB
:10115000800501FB12041B3C02D56442012000E023
:101160000020DFF898A080460027FA44AAF1BE0AC2
:101170000EE0E0070AD03246684607EB470101233C
:101180000AEB810100F022FB8DE8070064107F1C50
:10119000002CEED1194F7F44AE3F19E0E80715D07F
:1011A00007EB04100DF1180A90E80E008AE80E0013
:1011B000C068F04201D1981908903246012306A96F
:1011C00003A800F003FB03AB83E807006D10641C69
:1011D000002DE3D14FF0010332466946B8F1000F0C
:1011E00003A802D000F0DDFA01E000F0EFFAC9E94F
:1011F0000001C9F808200AB0BDE8F0878C5900004A
:1012000010B50446AFF300802046BDE81040FFF75C
:101210004CB8000000487047641300204FF0013CB8
:1012200050F8042B51F8043B9A4221D1A2EB0C0355
:10123000934313EACC1317D150F8042B51F8043B15
:101240009A4215D1A2EB0C03934313EACC130BD1B2
:1012500050F8042B51F8043B9A4209D1A2EB0C033D
:10126000934313EACC13DBD04FF00000704700BF6C
:10127000D01A01BAB1FA81F101F0180122FA01F095
:10128000CB40C1F12001DBB2C0B2C01A2CFA01F38D
:10129000D11A914311EAC311E6D1704701491820D0
:1012A000ABBEFEE72600020070475FEA400C08BFB5
:1012B00091F0000F4FEA8C234FEAC12243EA5151CB
:1012C0004FEA1C5018BF00F5F0404FEA300018BF3D
:1012D00041F000415FEA6C5C00F02980BCF1FF3F07
:1012E00008BF40F080407047130C06BF12044FF057
:1012F000100C4FF0000C130E04BF12020CF1080C7E
:10130000130F04BF12010CF1040C930F04BF9200E1
:101310000CF1020CD30F04BF52000CF1010C11466A
:101320004FF00002A0F11F00A0EB0C00704711F07D
:10133000004F08BF704731F000413FF4D5AF0B0CB0
:1013400006BF09044FF0100C4FF0000C0B0E04BF49
:1013500009020CF1080C0B0F04BF09010CF1040C7D
:101360008B0F04BF89000CF1020CCB0F04BF4900A6
:101370000CF1010CCCF12003A0EB0C0022FA03F3DA
:1013800002FA0CF241EA030100F10100704720F07B
:101390007F4C80EA030023F07F47ACEB070303F5A3
:1013A0007C5300F0004003F1FF032DE980494FEA30
:1013B000154B09B44FEA144325EA0B4E24EA0348BF
:1013C0000FF2042606EB132749083E785FEA320243
:1013D00003FB0667C7F5000707FB06F64FEA54371D
:1013E0004FEAD64606F1020607FB066CCCF1005C1C
:1013F0004FEA1C472CEA074C07FB06F40CFB06F5EA
:1014000004EB15464FEA961634BF00204FF000401B
:101410004FEAD13706FB07FC4FEA1C4C0CFB0BF7DD
:10142000D21B03FB0CF761EB07010CFB0EF7B0EBD3
:10143000074072EB17420CFB08F734BFA2EB0742E0
:10144000B2EB074261EB17414FEA0C444FEA9107B8
:1014500006FB07FC4FEA1C4C0CFB0BF7B0EBC7403C
:1014600072EB573203FB0CF734BFA2EBC742B2EB6F
:10147000C74261EB57310CFB0EF7B0EBC70072EBC4
:1014800057720CFB08F734BFA2EBC702B2EBC702DE
:1014900061EB5771039F4FEA816141EA921104EBBE
:1014A000CC044FEAD1374FEA826206FB07FC42EADE
:1014B00090124FEA80604FEA1C4C0CFB0BF7D21BDA
:1014C00003FB0CF761EB07010CFB0EF7B0EB0740D9
:1014D00072EB17420CFB08F734BFA2EB0742B2EBEA
:1014E000074261EB17414FEA8C554FEA910704EB35
:1014F0009C2406FB07FC4FEA1C4C0CFB0BF7B0EBE3
:10150000C74072EB573203FB0CF734BFA2EBC74264
:10151000B2EBC74261EB57310CFB0EF7B0EBC700E3
:1015200072EB57720CFB08F734BFA2EBC702B2EBA9
:10153000C70261EB577115EB4C254FEA816141EA17
:1015400092114FEA82624FEAD13742EA901206FBCB
:1015500007FC44F100044FEA80604FEA1C4C0CFB8E
:101560000BF7D21B03FB0CF761EB07010CFB0EF72B
:10157000B0EB074072EB17420CFB08F734BFA2EB4D
:101580000742B2EB074261EB174115EB1C154FEA1E
:10159000813141EA92414FEA823242EA90424FEA77
:1015A00080304FEA0C7644F1000448EA03434EEAE7
:1015B0000B484FF0000EB2EB080C71EB030724BF91
:1015C000624639464EEB0E0E4FF0000B00185241AA
:1015D00049414BEB0B0BB2EB080C71EB03077BF1B2
:1015E000000B24BF624639464EEB0E0E4FF0000B47
:1015F0000018524149414BEB0B0BB2EB080C71EB5D
:1016000003077BF1000B24BF624639464EEB0E0EFA
:1016100051EA020718BF46F0010616EB0E7655F1A7
:10162000000254F1000103D5BDE88901BDE800883E
:10163000BDE88901BDE80048B619524141EB0101FE
:10164000A3F10103704780807F7E7D7C7B7A79786F
:10165000777676757473727171706F6E6E6D6C6C77
:101660006B6A6A6968686766666564646363626119
:101670006160605F5F5E5E5D5D5C5C5B5B5A5A599A
:101680005958585757565655555554545353525206
:101690005251515050504F4F4F4E4E4D4D4D4C4C5E
:1016A0004C4B4B4B4A4A4A494949484848474747A7
:1016B00047464646454545444444444343434342E4
:1016C000424242414141002B9C4630D477002BD00E
:1016D0001CB54FEA370703B44FF010004FF010016C
:1016E000BAF1000F06D0BCF1000FDCBF40F00800DB
:1016F00040F008014FF000000FBCBDE810400BF1B6
:10170000010BBBF1010F08BF5FEA170722BF12F1FF
:10171000010211F101014FF0004143F1000300F01B
:10172000004043EA00007047F9D35708D0E746EA83
:10173000064613F1400F4FEA16461FDD13F1200F46
:10174000DFBF16430A46002120335B42BED0C3F1FF
:10175000200746EA064602FA07F74FEA164646EA27
:101760000706C3F1200722FA03F201FA07F721FA6C
:1017700003F14FF0000342EA0702A7E746EA020638
:1017800046EA06464FEA164646EA0106BCBF46EA66
:101790000646360C4FF000034FF000024FF00001F8
:1017A00094E72DE9804C9A46934670B491E838004E
:1017B00007C831EA400C48BF34EA430C03D5FFF7B1
:1017C000E6FDFFF780FFF0BCBDE8008C2DE9804C02
:1017D0009A46934670B491E8380007C810F0804FDD
:1017E00008BF13F0804F03D100F005F8FFF76BFF3F
:1017F000F0BCBDE8008C20F07F4780EA030023F0B6
:101800007F4C07EB0C03A3F57C5300F00040A3F1E1
:10181000FE0392F0000F00F0B38095F0000F00F08F
:1018200077802DE901494FEA11404FEA144621EA39
:10183000004800FB06FC24EA064708FB06F607FB07
:1018400008F800FB07F718EB06484CEB164C4FEA7C
:10185000124B18EB07484FEA15464CEB174022EAAB
:101860000B4E0BFB06FC25EA06470EFB06F607FBB4
:101870000EFE0BFB07F71EEB064E4CEB164C4FF023
:1018800000061EEB074E4CEB174B18EB0B0840F114
:10189000000018EB0E0B58EB000840F100008F1A07
:1018A0004FF000013CBFC943661B14BFB5EB040CED
:1018B00000213CBFC943F61B4FEA17444EEA8E0E87
:1018C00027EA04454FEA1C4704FB07622CEA074C51
:1018D00005FB07F70CFB05F604FB0CFC16EB0746B3
:1018E00042EB174216EB0C4642EB1C421BEB060682
:1018F00058EB0202414146EA9E0601D5BDE8018946
:10190000B619524141EB0101A3F10103BDE8018980
:101910004FEA14454FEA114724EA054621EA074CED
:1019200005FB07F406FB07F70CFB06F105FB0CFCB7
:1019300011EB074144EB17444FEA124711EB0C41FE
:1019400044EB1C4422EA074C05FB07F206FB07F7B1
:101950000CFB06F605FB0CFC16EB074642EB1742A8
:1019600016EB0C4642EB1C456A1854F1000148BFC7
:101970007047B619524141EB0101A3F101037047D1
:1019800095F0000F37D04FEA11424FEA144721EA91
:10199000024624EA074C02FB07F106FB07F70CFBA3
:1019A00006F402FB0CFC14EB074441EB17414FEA31
:1019B000154714EB0C4441EB1C4125EA074C02FB94
:1019C00007F506FB07F70CFB06F602FB0CFC16EB13
:1019D000074645EB174516EB0C4645EB1C42121922
:1019E00051F1000148BF7047B619524141EB010166
:1019F000A3F1010370474FEA14454FEA114724EA67
:101A0000054621EA074C05FB07F106FB07F70CFB2F
:101A100006F24FF0000605FB0CFC12EB074241EB0F
:101A2000174112EB0C4251EB1C4148BF7047921812
:101A300041EB0101A3F101037047000010B5002440
:101A4000384A1B21002000F081F8112035494870E8
:101A50004A1C0121084600F0B9F8022000F0BAFE45
:101A60000620304988708A1C0121022000F0AEF85F
:101A7000022000F0AFFE11202A49C870CA1C0121C3
:101A8000032000F0A3F8022000F0A4FE6020254906
:101A900008710A1D0121042000F098F8022000F0CE
:101AA00099FE40201F4948714A1D0121052000F080
:101AB0008DF8022000F08EFE45201A4988718A1D9B
:101AC0000121062000F082F8022000F083FE0920A8
:101AD0001449C87301F10F0201210F2000F076F8BC
:101AE000C82000F077FE192000F05AF8C82000F056
:101AF00071FE1B210B48FEF799FC0A4A1B210020AE
:101B000000F024F8022000F065FE082000F048F8FC
:101B100000200549086005A001F0AAFD05200A493A
:101B2000086010BDD00A0020900121424144533189
:101B30003236785F496E6974BAAFCAFDB3C9B9A6C7
:101B4000D6B4D0D00A000000100000202DE9F041EA
:101B500006460C46174600201049086000BF00BF2B
:101B600000BF00BF00BF00BF00BF00BF06F12001E3
:101B7000C8B202F08DFB611EC8B202F089FB0025DD
:101B800004E0002002F084FB78556D1CA542F8D3D8
:101B9000012002490860BDE8F08100009001214267
:101BA00070B50446002008490860204602F070FB2A
:101BB0000546012004490860192C03D14FF47A70BE
:101BC00000F008FE00BF70BD900121422DE9F041F8
:101BD00006460C46154600201449086000BF00BFA9
:101BE00000BF00BF00BF00BF00BF00BF06F1400143
:101BF000C8B202F04DFB611EC8B202F049FB00BF43
:101C000000BF00BF00BF00BF00BF00BF00BF002774
:101C100004E015F8010B02F03BFB7F1CA742F8D350
:101C2000012002490860BDE8F081000090012142D6
:101C300030B5024600201FE000EB4003104C04EBDF
:101C4000C3031B69934216D100EB400354F83330B1
:101C500083B9012300EB4004094D45F8343000EB13
:101C600040032C4604EBC303D96000EB400304EBB4
:101C7000C303996002E0401C0C28DDD300BF30BDD7
:101C8000AC00002030B50546074805600120074933
:101C900008700748448CC82C00DAC824214602206A
:101CA000FFF7C6FF30BD0000DC010020D801002096
:101CB000EC0A002000BFFEE70021114A82F82E1036
:101CC00011869163D163116451649164D16482F887
:101CD0005010002005E000220949543141F820202D
:101CE000401C1E28F7DB0021054A82F82D1082F8DF
:101CF000CC1082F8CD1082F8CE1082F8CF10704749
:101D0000EC0A002070B5114D002400F095FB00BFD7
:101D100000BF0F4802782146641C6A540C222146F9
:101D2000641C6A5401222146641C6A5490F82E20D7
:101D30002146641C6A542946204601F089FC285536
:101D4000601C0449087002F0DFFA70BDD40B00205B
:101D5000EC0A00205500002070B5114D002400F061
:101D6000D7FB00BF00BF0F4802782146641C6A54AD
:101D70000B222146641C6A5401222146641C6A54C9
:101D800090F82E202146641C6A542946204601F012
:101D90005FFC2855601C0449087002F0B5FA70BD5C
:101DA000D40B0020EC0A00205500002070B5144E22
:101DB000144D0024F07810B100F01CFC01E002F09A
:101DC000FDFC104D0024104802782146641C6A5422
:101DD0000D222146641C6A5401222146641C6A5467
:101DE00090F82E202146641C6A542946204601F0B2
:101DF0002FFC2855601C0549087002F085FA70BD5B
:101E0000D40C0020D40B0020EC0A00205500002048
:101E100070B5114D002400F013FC00BF00BF0F4847
:101E200002782146641C6A540A222146641C6A54C2
:101E300001222146641C6A5490F82E202146641C1D
:101E40006A542946204601F003FC2855601C0449C9
:101E5000087002F059FA70BDD40B0020EC0A002083
:101E60005500002070B5124D00240120114981F861
:101E70002D0000BF00BF084602782146641C6A544A
:101E800010222146641C6A5401222146641C6A54B3
:101E900090F82E202146641C6A542946204601F001
:101EA000D7FB2855601C0449087002F02DFA70BD5C
:101EB000D40B0020EC0A00205500002070B5154D11
:101EC000002415480079154981F82C00124A11792F
:101ED000D07802F0B5FA00BF00BF10480278214662
:101EE000641C6A540E222146641C6A540122214655
:101EF000641C6A5490F82E202146641C6A542946BA
:101F0000204601F0A5FB2855601C0549087002F029
:101F1000FBF970BDD40B0020D40C0020EC0A00208B
:101F20005500002070B5124D002401F065FB00F053
:101F3000EFFA00BF00BF0F4802782146641C6A54C4
:101F40000F222146641C6A5401222146641C6A54F3
:101F500090F82E202146641C6A542946204601F040
:101F600077FB2855601C0449087002F0CDF970BD5C
:101F7000D40B0020EC0A0020550000202DE9F04190
:101F80002C4C2079E17800EB01202B49C882A07904
:101F9000617900EB012028490883207AE17900EB80
:101FA000012025494883607A0877A07A4877E07A4B
:101FB0008877607B217B00EB01201F490884E07B50
:101FC000A17B00EB01201C494884277C3804617CFC
:101FD00000EB0120A17C084417494862E77C3804E3
:101FE000217D00EB0120617D0844134988620320B4
:101FF000FFF748FE114E00250F48027829466D1C58
:102000007254082229466D1C7254012229466D1C07
:10201000725490F82E2029466D1C72543146284681
:1020200001F016FB7055681C0549087002F06CF948
:10203000BDE8F081D40C0020EC0A0020D40B002075
:102040005500002070B56B4D00246B480278214686
:10205000641C6A5411222146641C6A54641C90F862
:102060002E202146641C6A54806BC0F3074221462F
:10207000641C6A546048008FC0F307222146641C28
:102080006A545D4890F838202146641C6A54C06B3D
:10209000C0F307422046611CCCB22A545648808FB8
:1020A000C0F307222046611CCCB22A54524890F853
:1020B0003C202046611CCCB22A544F48006CC0F32F
:1020C00007422046611CCCB22A544B48B0F840006D
:1020D000C0F307222046611CCCB22A54464890F82F
:1020E00040202046611CCCB22A544348406CC0F3C7
:1020F00007422046611CCCB22A543F48B0F8440045
:10210000C0F307222046611CCCB22A543A4890F80A
:1021100044202046611CCCB22A543748806CC0F35E
:1021200007422046611CCCB22A543348B0F848001C
:10213000C0F307222046611CCCB22A542E4890F8E6
:1021400048202046611CCCB22A542B48C06CC0F3F6
:1021500007422046611CCCB22A542748B0F84C00F4
:10216000C0F307222046611CCCB22A54224890F8C2
:102170004C202046611CCCB22A541F4890F85020B5
:102180002046611CCCB22A54002620E0FE2E00DB43
:1021900022E01948543050F82600C0F30742204688
:1021A000611CCCB22A541448543030F82600C0F3D5
:1021B00007222046611CCCB22A540F48543010F834
:1021C00026202046611CCCB22A54701CC6B20A4894
:1021D00090F85000B042D9DC00BFE01EA87029463C
:1021E000204601F035FA2855601C0449087002F0B9
:1021F0008BF870BDD40B0020EC0A002055000020A5
:1022000070B52C4D00242C4802782146641C6A5479
:1022100009222146641C6A54641C90F82E20214631
:10222000641C6A5490F8CC202146641C6A5490F8CF
:10223000CD202146641C6A5490F8CE202146641CAF
:102240006A5490F8CF202046611CCCB22A541A4818
:10225000008E020A2046611CCCB22A54164890F81F
:1022600030202046611CCCB22A541348406BC0F386
:1022700007422046611CCCB22A540F48808EC0F31E
:1022800007222046611CCCB22A540B4890F8342017
:102290002046611CCCB22A54E01EA8702946204674
:1022A00001F0D6F92855601C0449087002F02CF89A
:1022B00070BD0000D40B0020EC0A00205500002067
:1022C00070B5104D002400BF00BF0F4802782146B2
:1022D000641C6A5407222146641C6A540122214668
:1022E000641C6A5490F82E202146641C6A542946C6
:1022F000204601F0ADF92855601C0449087002F031
:1023000003F870BDD40B0020EC0A0020550000201B
:1023100070B5154D0024154802782146641C6A5496
:1023200001222146641C6A54641C90F82E20214628
:10233000641C6A5428190D49491CFDF7EFFF0B482E
:10234000401CFEF70FF8401C2044C4B2E01EA870E9
:102350002946204601F07CF92855601C0449087084
:1023600001F0D2FF70BD0000D40B0020EC0A002069
:102370005500002070B5134D00241348C678304630
:1023800001F0AEFF114802782146641C6A54022213
:102390002146641C6A542146641C6A5490F82E201D
:1023A0002146641C6A542146641C6E54294620460A
:1023B00001F04EF92855601C0549087001F0A4FF92
:1023C00070BD0000D40B0020D40C0020EC0A0020CB
:1023D0005500002070B5144E144D0024F07810B153
:1023E00000F0A6F901E002F05BFA104D002410485D
:1023F00002782146641C6A5412222146641C6A54E5
:1024000001222146641C6A5490F82E202146641C47
:102410006A542946204601F01BF92855601C0549DD
:10242000087001F071FF70BDD40C0020D40B0020A7
:10243000EC0A00205500002008B51D4890F8CD009A
:1024400000F0040000B108BD01201A4908601A48D4
:10245000006840F04000184908600846006820F015
:10246000200008600846008814490880104890F849
:10247000CD0040F004000E4981F8CD0000BF10A04F
:10248000104BD02210A1009013A001F0F1F81DA074
:1024900000900748408B4FF47A7100FB01F21B4B10
:1024A0000121002002F09CF800BF00BFCBE7000034
:1024B000EC0A0020A88121424C0000202C000020C2
:1024C00030000000A06900084170705C4945445F1D
:1024D0004354524C2E43000046696C6520257320FE
:1024E000204C696E65202564202573205374617229
:1024F0007454696D6572576974684E616D652825FD
:102500007329000053746F7044480000BD460008F2
:1025100008B5204890F8CD0000F0020028B91D4809
:1025200090F8CD0000F0010000B108BD01201A496B
:1025300008601A48006840F0020018490860084620
:10254000006820F0010008600846008814490880EF
:10255000104890F8CD0040F002000E4981F8CD00FF
:1025600000BF10A0104BAA2210A1009013A001F0F0
:102570007FF81DA000900748008B4FF47A7100FB94
:1025800001F21B4B0121002002F02AF800BF00BF1E
:10259000CBE70000EC0A0020808121424C000020A3
:1025A0002C000020300000008F6900084170705C32
:1025B0004945445F4354524C2E43000046696C65C4
:1025C00020257320204C696E65202564202573200A
:1025D000537461727454696D6572576974684E61A1
:1025E0006D6528257329000053746F7046530000F1
:1025F000714700080E4890F8CD0000F0080000B1C7
:10260000704701200B4908600B48006840F010003B
:10261000094908600846008808490880044890F87D
:10262000CD0040F00800024981F8CD0000BFE7E787
:10263000EC0A0020888121424C0000202C00002060
:1026400008B5204890F8CD0000F0010028B91D48D9
:1026500090F8CD0000F0020000B108BD1A480088D3
:102660001A49088000BF1AA01C4B85221CA10090AB
:102670001FA000F0FDFF29A000901248C08A4FF46F
:102680007A7100FB01F2274B0121274801F0A8FFD6
:1026900000BF25480068002810DB0120234908609E
:1026A0000948006840F0080007490860054890F8AC
:1026B000CD0040F00100034981F8CD0002F0F0F8B0
:1026C00000BFCAE7EC0A00204C0000202C000020CC
:1026D0002654696D65724A53000000008569000840
:1026E0004170705C4945445F4354524C2E43000096
:1026F00046696C6520257320204C696E6520256431
:1027000020257320537461727454696D6572576922
:1027100074684E616D6528257329000053746F70CD
:102720004A530000F94700084800002084812142F4
:1027300008B50D480068401C002814D101200B4941
:10274000086000BF0AA00E4B58220EA1009011A0F5
:1027500000F08EFF1AA01C4B1C4A01210090024879
:1027600001F03EFF00BF08BD44000020940122425A
:102770002654696D657253746F70574A42000000A9
:10278000736900084170705C4945445F4354524C82
:102790002E43000046696C6520257320204C696E2D
:1027A0006520256420257320537461727454696D0B
:1027B0006572576974684E616D652825732900003C
:1027C00053746F7058484200A1480008C0270900A0
:1027D0007047000030B501464FF0E0246269114CAB
:1027E00024684FF4FA55B4FBF5F301FB03F4641EBF
:1027F0004FF0E0256C610024AC612C46246944F064
:1028000001042C6100BF4FF0E024206900F00104B6
:102810001CB100F48034002CF5D04FF0E02462614C
:1028200030BD00008400002001460888704770B564
:1028300004460D462946204600F022FA70BD0000ED
:1028400070B505460B4614462E465B080648044400
:10285000002206E004EB4200FFF7E6FF26F8120034
:10286000521C9A42F6D370BD00F0000810B5044621
:10287000E00AC402204600F087F910BD2DE9F04FB0
:1028800085B082460F4616460020049037480290D5
:1028900078080190F00A354901EBC029C6F30A0611
:1028A000B819C0F30A0008B1012000E00020B919EE
:1028B00000EBD12BC6F3490000900024A04625462A
:1028C000039403A800F049FA039818B9049805B0D6
:1028D000BDE8F08F002544E000240BE04FF40061D8
:1028E00001FB059101EB4400FFF79EFF204921F811
:1028F0001400641CB4F5806FF0D30DB9009800E0AB
:10290000002004460DE03AF81800194921F8140097
:102910000198401E019008B900BF05E0641C08F151
:102920000108B4F5806FEED300BF00F0F7F909EBB2
:10293000C520FFF79BFF00240BE04FF4006202FB71
:10294000059202EB44000A4A32F81410FFF76FFFB9
:10295000641CB4F5806FF0D300F088F9FF20049078
:102960006D1C5D45B8D30498B1E7000000F0000885
:10297000E401002010B501F003F8012005490860CA
:1029800005480068801105494863402000F008F8B8
:1029900010BD000010000020C40A0020EC0A002036
:1029A00010B50446200D000508B904B103E0FC2170
:1029B00002A003F071FE1048046010BD4C69627201
:1029C00061726965735C53544D3332463130785FC0
:1029D0005374645065726970685F44726976657299
:1029E0005C7372635C73746D3332663130785F652B
:1029F0007874692E630000001404014070B5044629
:102A00000025207910B12079042800D103E06A2143
:102A100035A003F041FE6079082805D060790C28C4
:102A200002D06079102800D103E06B212EA003F0C2
:102A300033FE20686FF3130010B9206800B103E083
:102A40006C2129A003F028FEA07910B1A0790128FB
:102A500000D103E06D2124A003F01EFE314DA079CA
:102A600090B3284600682168884329460860081DFD
:102A7000006821688843291D08602079054428687A
:102A80002168084328602748083000682168884387
:102A9000244908310860081D0068216888432149DD
:102AA0000C310860607910280FD1081F0068216878
:102AB00008431C4908310860081D00682168084364
:102AC00018490C3108600EE007E0164D60790544A6
:102AD000286821680843286005E0207905442868B3
:102AE00021688843286070BD4C69627261726965B3
:102AF000735C53544D3332463130785F53746450B5
:102B000065726970685F4472697665725C7372633E
:102B10005C73746D3332663130785F657874692E1A
:102B2000630000000004014010B5044624F03500A5
:102B300008B904B104E040F2B65103A003F0ACFDC3
:102B40001048C46010BD00004C6962726172696512
:102B5000735C53544D3332463130785F5374645054
:102B600065726970685F4472697665725C737263DE
:102B70005C73746D3332663130785F666C61736894
:102B80002E6300000020024070B504460425B4F115
:102B9000006F03D31448844200D204E040F2A7112E
:102BA00012A003F079FD4FF4302000F0C3F8054681
:102BB000042D17D11C48006940F002001A49086131
:102BC00008464461006940F0400008614FF430203D
:102BD00000F0B0F805461448006941F6FD71084060
:102BE00011490861284670BDFFFF0F084C696272E9
:102BF00061726965735C53544D3332463130785F8E
:102C00005374645065726970685F44726976657266
:102C10005C7372635C73746D3332663130785F66F7
:102C20006C6173682E6300000020024004200B4991
:102C3000C96801F0010109B101200EE00749C96826
:102C400001F0040109B1022007E00449C96801F05C
:102C5000100109B1032000E0042070470020024069
:102C60000148006A704700000020024003480069E4
:102C700040F08000014908617047000000200240D8
:102C800070B504460D460426B4F1006F03D3124814
:102C9000844200D204E040F25E3110A003F0FCFC5C
:102CA0004FF4005000F046F80646042E11D11A48A1
:102CB000006940F00100184908612580F00200F029
:102CC00039F806461448006941F6FE710840124979
:102CD0000861304670BD0000FFFF0F084C6962724A
:102CE00061726965735C53544D3332463130785F9D
:102CF0005374645065726970685F44726976657276
:102D00005C7372635C73746D3332663130785F6606
:102D10006C6173682E630000002002400248034982
:102D2000486003484860704723016745002002401F
:102D3000AB89EFCD00B502460423FFF777FF0346CA
:102D400003E0FFF773FF0346521E012B01D1002A57
:102D5000F7D102B90523184600BD38B50446352021
:102D6000FFF7E2FEFFF77CFF0090009800F0C00044
:102D7000206038BD70B505460C4600265DB1012DBA
:102D800009D0022D07D0032D05D0042D03D0052D29
:102D900001D0062D00D104E040F2652121A003F00E
:102DA0007BFCECB1012C1BD0022C19D0032C17D0CA
:102DB000042C15D0052C13D0062C11D0072C0FD0C5
:102DC000082C0DD0092C0BD00A2C09D00B2C07D0C5
:102DD0000C2C05D00D2C03D00E2C01D00F2C00D1C3
:102DE00004E040F266210FA003F056FCA007010F9B
:102DF0000F2000FA01F61A48A11050F82100B04344
:102E00001749A21041F822000846A11050F82100ED
:102E1000A107090F05FA01F108431149A21041F871
:102E2000220070BD4C69627261726965735C5354B3
:102E30004D3332463130785F537464506572697037
:102E4000685F4472697665725C7372635C73746DFB
:102E50003332663130785F6770696F2E630000002F
:102E6000080001402DE9F05F05460C464FF00009CF
:102E7000CA4600260027B046B3465948854211D0BD
:102E8000584885420ED0584885420BD05748854255
:102E900008D05748854205D05648854202D056484A
:102EA000854200D103E0B22154A003F0F5FBE078A5
:102EB000A0B1E078042811D0E07828280ED0E0787E
:102EC00048280BD0E078142808D0E078102805D0E6
:102ED000E0781C2802D0E078182800D103E0B32164
:102EE00046A003F0D9FB002010B9208800B103E010
:102EF000B42142A003F0D0FBE07800F00F09E078A5
:102F000000F0100080B1A078012805D0A078022838
:102F100002D0A078032800D103E0BB2137A003F042
:102F2000BBFBA07840EA0909207838B3D5F80080C7
:102F300000261FE0012000FA06F7208800EA070AB1
:102F4000BA4516D1B7000F2000FA07FB28EA0B0894
:102F500009FA07F040EA0808E078282803D10120A0
:102F6000B040686105E0E078482802D10120B04017
:102F70002861761C082EDDD3C5F800802088FF2844
:102F80002BDDD5F80480002623E006F1080001219E
:102F900001FA00F7208800EA070ABA4518D1B700FD
:102FA0000F2000FA07FB28EA0B0809FA07F040EAAD
:102FB0000808E078282803D106F1080081406961FB
:102FC000E078482804D106F10800012181402961F8
:102FD000761C082ED9D3C5F80480BDE8F09F000008
:102FE00000080140000C01400010014000140140A5
:102FF00000180140001C0140002001404C69627231
:1030000061726965735C53544D3332463130785F79
:103010005374645065726970685F44726976657252
:103020005C7372635C73746D3332663130785F67E2
:1030300070696F2E630000002DE9F04704460E46CC
:103040000027B8460025A946012C7DD0022C7BD054
:10305000042C79D0082C77D0694884427FD0684806
:10306000203084427BD06748844278D065488030E5
:10307000844274D06448844271D0644884426ED0E3
:10308000634884426BD06348844268D0624884427B
:1030900065D0B4F5805F62D0B4F5EA1F5FD0B4F5B7
:1030A000EB1F5CD0B4F5004F59D05C48844256D039
:1030B000401C844253D0801C844250D0001D844266
:1030C0004DD056480F30844249D0B4F1201F46D02D
:1030D0004FEAF030844242D0514884423FD05148B8
:1030E00084423CD05048844239D05048844236D043
:1030F0004F48844233D0B4F5011F30D04D4884424C
:103100002DD0401C84422AD0801C844227D0001D30
:10311000844224D047480F30844220D045481F3095
:1031200084421CD043483F30844218D041487F300D
:10313000844214D03F48FF30844210D03E4884423D
:103140000DD03E48844200E009E008D03C4884426B
:1031500005D03C48844202D03B48844200D104E080
:1031600040F22A2139A003F097FA0EB1012E00D1C6
:1031700004E040F22B2135A003F08EFA04F0004069
:10318000B0F1004F02D14048C56901E03E484568B2
:10319000C4F30349A7B204F44010B0F5401F08D1AE
:1031A00025F070653848406820F070603649486006
:1031B00013E004F48010B0F5801F07D1032000FA5B
:1031C00009F825EA080545F0706506E0600D000184
:1031D00007FA00F0854345F0706526B1600D0101E6
:1031E00007FA01F0054304F00040B0F1004F02D1AE
:1031F0002548C56101E024484560BDE8F08700002E
:103200001000140040001600000118000002180011
:103210000003180000081A00000C1A00010020002A
:1032200000013000000230000004300000112000D6
:1032300000202000010000800002008000040080C7
:103240000008008000100080002000804C6962723D
:1032500061726965735C53544D3332463130785F27
:103260005374645065726970685F44726976657200
:103270005C7372635C73746D3332663130785F6790
:1032800070696F2E6300000000000140FEB5054626
:10329000002000900190029000241E49086000F078
:1032A000F7FF0646002000F0F3FF0443240200204D
:1032B00000F0EEFF04432402002000F0E9FF044385
:1032C0002402002000F0E4FF0443002000F0E0FFAF
:1032D0000746201E01DB014600E0414200910197B4
:1032E000029600BF00BF00BF00BF00BF00BF00BF0D
:1032F00000BF00BF00BF00BF00BF00BF00BF00BFD6
:1033000000BF0120034908609DE8070085E8070029
:10331000FEBD0000900121420B4909780B4A12784A
:1033200091420ED00A49084A1278885C0649097809
:10333000491C0A2291FBF2F302FB1311024A11709D
:1033400000E0002070470000810000208000002085
:10335000D40D00200148006870470000D40100200F
:1033600000BFFEE710B500F041F80120FFF732FA88
:1033700072B60620FEF714FC1420FFF72BFAFEF7B6
:103380005DFB62B610BD000000200549C86005491C
:1033900008600549086005490860054908607047EC
:1033A000001001400C0801400C0C01400C140140BD
:1033B0000C18014010B503F073F9D4210848FDF74B
:1033C00035F808A10648401CFCF7A8FF0120044975
:1033D000087000F0BDFA0020014981F8D00010BD4E
:1033E000EC0A002048585F4C525931000EB51720A6
:1033F0008DF8080002208DF809008DF80A000120E0
:103400008DF80B0002A800F04BF906210020FFF711
:10341000B1FC4020009000208DF804000C208DF8B5
:10342000050001208DF806006846FFF7E7FA0EBD9B
:1034300010B500F001F810BD00B587B0B020ADF8B0
:10344000040003208DF8060010208DF8070001A964
:103450002348FFF707FD4020ADF8040004208DF855
:10346000070001A91E48FFF7FDFCA020ADF80400ED
:1034700018208DF8070001A91948FFF7F3FC012077
:10348000184908600121000300F0B2F90021012071
:10349000FFF7D2FD0020ADF808004FF48270ADF8C0
:1034A0000A000020ADF80C00ADF80E000120ADF8C8
:1034B00010004002ADF812002020ADF814000020EA
:1034C000ADF816000720ADF8180002A9064800F074
:1034D00017FE0121044800F001FD07B000BD000007
:1034E00000080140900121420030014000B587B042
:1034F000012144F2010000F07BF94FF48060ADF847
:10350000040004208DF8070001A92F48FFF7AAFC4A
:103510004FF40070ADF8040003208DF80600182069
:103520008DF8070001A92848FFF79CFC4FF41650BE
:1035300003900020ADF81000ADF81200ADF81400B3
:10354000ADF818000C20ADF8160003A91F4802F0D2
:1035500091FD4FF4E06000F011F90B208DF80800A8
:1035600001208DF80A0000208DF8090001208DF857
:103570000B0002A800F094F825208DF8080002A89E
:1035800000F08EF8012240F22551104802F0CEFCE6
:1035900001210E4802F0CEFB00200D4908600D49C4
:1035A00008700D4908700D4908700D4908700D49E3
:1035B00008600D4908600D4908600D4908600D4913
:1035C000086007B000BD000000080140003801405D
:1035D000A001214255000020540000205600002088
:1035E000570000205C0000206000002064000020E4
:1035F000680000207000002010B501F02FF80920AD
:1036000001F08CF9082001F089F90A2001F086F90F
:103610000B2001F083F901F051F801F0CFF801F02F
:10362000EBF8FEF749FB0020014981F8D00010BDFE
:10363000EC0A002070470000044890F8CD0020F00C
:103640000400024981F8CD0070470000EC0A002018
:1036500010B502460B46FF20002103E05C5C604091
:103660004C1CE1B29142F9DB10BD00BFFEE7000047
:103670000FB438B5002405A800900748009A0499B3
:10368000FCF73AFE044600200090034900F00CFBD2
:10369000204638BC5DF814FB301300207047000052
:1036A0002DE9F0410446002500270F26E07810B1EF
:1036B000E078012800D103E0752121A002F0ECFFA1
:1036C0006078102800DA03E076211DA002F0E4FF04
:1036D000A078102800DA03E0772119A002F0DCFFBF
:1036E000E07800B32248006800F4E060C0F5E060D4
:1036F000050AC5F10407EE40607800FA07F5A078E6
:10370000304005432D011B4822788554207800F075
:103710001F010120884021784911890001F1E02131
:10372000C1F8000109E0207800F01F010120884065
:1037300011492278521141F82200BDE8F0810000C1
:103740004C69627261726965735C53544D333246E1
:103750003130785F5374645065726970685F447289
:10376000697665725C7372635C6D6973632E630066
:103770000CED00E000E400E080E100E010B504465C
:10378000B4F5E06F0BD0B4F5C06F08D0B4F5A06FFE
:1037900005D0B4F5806F02D0B4F5407F00D103E0CE
:1037A000632104A002F078FF0E4820430E49086010
:1037B00010BD00004C69627261726965735C53549C
:1037C0004D3332463130785F53746450657269709E
:1037D000685F4472697665725C7372635C6D69736D
:1037E000632E63000000FA050CED00E07047000056
:1037F00070B504460D461048204008B904B104E0F5
:1038000040F24A410DA002F047FF0DB1012D00D159
:1038100004E040F24B4109A002F03EFF2DB11648F2
:10382000806920431449886104E013488069A043FB
:103830001149886170BD00000200C0FF4C696272CE
:1038400061726965735C53544D3332463130785F31
:103850005374645065726970685F4472697665720A
:103860005C7372635C73746D3332663130785F728F
:1038700063632E63000000000010024030B5002199
:103880000022002400232D4D6D6805F00C0121B1AC
:10389000042905D0082923D105E0294D056022E03F
:1038A000274D05601FE0254D6D6805F47012234D0E
:1038B0006D6805F48034022505EB92421CB9214D58
:1038C000554305600BE01D4D6D6805F400351DB1D5
:1038D0001C4D5543056002E0194D5543056002E05B
:1038E000174D056000BF00BF144D6D6805F0F00175
:1038F0000909154D6B5C0568DD4045600F4D6D682D
:1039000005F4E061090A104D6B5C4568DD40856097
:103910000A4D6D6805F46051C90A0B4D6B5C456832
:10392000DD40C560054D6D6805F44041890B074DCC
:103930006B5CC568B5FBF3F5056130BD0010024056
:1039400000127A0000093D0098000020A800002025
:1039500000B5002204210848FEF772FF06480078EF
:10396000552804D1044840780449087002E0FF203B
:103970000249087000BD000000000020EC0A002091
:103980003EB5002400256846FFF780FC23489DE8EB
:103990000E000EC0224801680068401C204A1060DA
:1039A00001EB41001F4901EB80001C4B0ECB0EC008
:1039B0001B490868C11700EB11710911A0EB011137
:1039C000174A11601548006801121748026800681C
:1039D000401C154B1860154840F82210194608681D
:1039E000C11700EB5171C910A0EBC1011A4611605B
:1039F00001200F4908600D480568012409E00B48C3
:103A000050F82400A84203D000200949086002E0D1
:103A1000641C082CF3DB00BF3EBD0000C40A00207C
:103A200004000020E409002008000020A40A00206F
:103A30000C0000200548406B0449C863084690F814
:103A4000CE0040F0020081F8CE007047EC0A002062
:103A50000548406B04494864084690F8CE0040F0A1
:103A6000080081F8CE007047EC0A002038B52148E4
:103A700090F85000022827DD1E4890F85000401EA4
:103A80001C49543151F820005439496B451A1948E2
:103A9000846AA54218DB406B16498864084690F892
:103AA000CE0040F0200081F8CE0000BF12A0164BDF
:103AB00040F2511215A1009018A0FFF7D9FD20483F
:103AC00002F018FD00BF38BD0A4890F850001E28CB
:103AD0000DDA0848416B90F8502090F85000401CD7
:103AE000044B83F8500003F1540040F8221000BF4B
:103AF000E9E70000EC0A0020266763526561645420
:103B00006954696D65720000AA6900084170705CB3
:103B10004945445F4354524C2E43000046696C654E
:103B200020257320204C696E652025642025732094
:103B300053746F7054696D657228257329000000F5
:103B4000300000200548406B0449C864084690F8DE
:103B5000CE0040F0400081F8CE007047EC0A002013
:103B60000548406B04490864084690F8CE0040F0D0
:103B7000040081F8CE007047EC0A00200548406B35
:103B800004498863084690F8CE0040F0010081F8AF
:103B9000CE007047EC0A00200548406B0449886459
:103BA000084690F8CE0040F0200081F8CE00704723
:103BB000EC0A002010B500BF0748007808B902F0F1
:103BC00067FB00BF05A0FFF753FD08A0FFF750FDFE
:103BD00006A0FFF74DFD10BDB8120020525454202E
:103BE0005072696E7466210A000000000A0000002D
:103BF0002DE9F04104460D46164600BF08480078FE
:103C000008B902F045FB00BF00BF324629462046F6
:103C100000F008F8074600BF3846BDE8F081000014
:103C2000B81200202DE9F047074688461646C246DE
:103C300007EB47011B4800EBC109D9F8140020B17C
:103C4000012811D0022826D11EE0484602F058FB78
:103C50000546B54201D2002405E0344632465146BD
:103C6000484602F0D8FC18E0484602F049FB0546F9
:103C7000B54201D2284600E030460446224651466D
:103C8000484602F0C8FC08E032465146484602F079
:103C900089FC044601E0002400BF00BF2046BDE8C7
:103CA000F0870000D01200200FB438B5044606A8F3
:103CB00000906A462046059900F003F838BC5DF88C
:103CC00014FB2DE9F04F99B082460D46144603A827
:103CD00014904020159000201690CDF860A0179009
:103CE00000BF95F900606D1C06B9E3E0252E73D185
:103CF00000274FF0010900BF95F90060232E12D074
:103D00002B2E0CD02D2E02D0302E10D103E047F0F8
:103D100001076D1C0EE047F002076D1C0AE047F03A
:103D200004076D1C06E047F008076D1C02E04FF029
:103D3000000900BF00BFB9F1000FDDD14FF000084E
:103D400000BF95F90060302E01DB392E00DD07E061
:103D50006D1CA6F1300008EB880100EB4108F0E78C
:103D600000BF0020139095F900602E2E13D16D1C1A
:103D700000BF95F90060302E01DB392E00DD09E02F
:103D80006D1CA6F13000139901EB810100EB41009D
:103D90001390EEE700BF95F9006000BF6C2E01D0D4
:103DA000682E03D195F900606D1C00E000E0F5E796
:103DB00000BF702E5DD008DC252E6AD0582E35D07D
:103DC000632E0AD0642E69D113E0732E3CD0752E79
:103DD0001DD0782E62D128E064E02168081D2060A3
:103DE000D1F800904FFA89FB594614A802F0B8FBAD
:103DF00055E02168081D2060D1F80090CDE90087CA
:103E00000A22494614A8139B02F088FA47E0216869
:103E1000081D2060D1F80090CDE900870A224946AC
:103E200014A8139B02F0F0FA39E000BF2168081DC6
:103E30002060D1F80090CDE900871022494614A8EF
:103E4000139B02F0E1FA2AE02168081D2060D1F8F6
:103E500000B000BF9BF900600BF1010B06B906E052
:103E6000314614A802F07CFB17980028F2DA00BF54
:103E700015E02168081D2060D1F80090002008217D
:103E80000B461022CDE90010494614A802F0BCFAF6
:103E900005E0252114A802F063FB00E000BF00BF8D
:103EA0006D1C03E0314614A802F05AFB1798002855
:103EB000BFF617AF00BF179800280ADD169820B18B
:103EC00003A95046169AFFF793FEDDE91610084441
:103ED0001790179819B0BDE8F08F000070B5044630
:103EE0000D461248844205D01148844202D0114840
:103EF000844200D104E04FF4D7710FA002F0CCFB54
:103F00000DB1012D00D104E040F2AF110AA002F082
:103F1000C3FB25B1208840F04000208004E02088C9
:103F20004FF6BF710840208070BD00000030014096
:103F300000380040003C00404C6962726172696563
:103F4000735C53544D3332463130785F5374645050
:103F500065726970685F4472697665725C737263DA
:103F60005C73746D3332663130785F7370692E63C1
:103F70000000000070B505460C4600261648854234
:103F800005D01648854202D01548854200D104E08C
:103F900040F2023113A002F07FFB802C0DD0402CA8
:103FA0000BD0202C09D0102C07D0082C05D0042CC5
:103FB00003D0022C01D0012C00D104E040F20331E7
:103FC00008A002F069FB2889204008B1012600E022
:103FD0000026304670BD000000300140003800402F
:103FE000003C00404C69627261726965735C5354B5
:103FF0004D3332463130785F537464506572697066
:10400000685F4472697665725C7372635C73746D29
:104010003332663130785F7370692E6300000000C0
:1040200010B504460848844205D00848844202D0AE
:104030000748844200D104E040F2362105A002F096
:104040002BFBA08910BD000000300140003800406B
:10405000003C00404C69627261726965735C535444
:104060004D3332463130785F5374645065726970F5
:10407000685F4472697665725C7372635C73746DB9
:104080003332663130785F7370692E630000000050
:1040900070B504460D460848844205D0074884425E
:1040A00002D00748844200D104E040F2262105A056
:1040B00002F0F2FAA58170BD0030014000380040E6
:1040C000003C00404C69627261726965735C5354D4
:1040D0004D3332463130785F537464506572697085
:1040E000685F4472697665725C7372635C73746D49
:1040F0003332663130785F7370692E6300000000E0
:1041000070B505460C4600264F48854205D04F48FD
:10411000854202D04E48854200D103E0A3214DA044
:1041200002F0BAFA208858B12088B0F5806F07D025
:104130002088B0F5004F03D02088B0F5404F00D163
:1041400003E0A62143A002F0A7FA6088B0F5827FC1
:1041500001D0608800B903E0A7213EA002F09CFADC
:10416000A088B0F5006F01D0A08800B903E0A821B5
:1041700038A002F091FAE08810B1E088022800D15E
:1041800003E0A92133A002F087FA208910B1208929
:10419000012800D103E0AA212EA002F07DFA608957
:1041A000B0F5007F01D0608900B903E0AB2129A000
:1041B00002F072FAA089A0B1A089082811D0A089C4
:1041C00010280ED0A08918280BD0A089202808D04C
:1041D000A089282805D0A089302802D0A0893828B5
:1041E00000D103E0AC211BA002F056FAE08910B127
:1041F000E089802800D103E0AD2116A002F04CFA3E
:10420000208A012800DB03E0AE2112A002F044FA6C
:104210002E8806F44156208861880843A188084307
:10422000E18808432189084361890843A18908433B
:10423000E189084306432E80A88B4FF2FF710840A6
:10424000A883208A288270BD0030014000380040D9
:10425000003C00404C69627261726965735C535442
:104260004D3332463130785F5374645065726970F3
:10427000685F4472697665725C7372635C73746DB7
:104280003332663130785F7370692E63000000004E
:1042900070B50446002500BF00BF00BF00BF00BFCF
:1042A00000BF00BF00BF00BF02210B48FFF762FE46
:1042B0000028F9D021460848FFF7EAFE00BF012197
:1042C0000548FFF757FE0028F9D00348FFF7A8FE7E
:1042D000C5B2284670BD00000030014070470000A4
:1042E00038B5044606A0006800908DF80140002211
:1042F00004216846FEF7C2FA0248047038BD000087
:1043000055000000EC0A002000200B4908700B4902
:10431000087001200A4908600A49086002200A4919
:1043200008600120094908604FF4FA7008490860E4
:104330000020084908607047540000205700002002
:10434000A0012142600000206400002068000020DD
:104350006C0000207000002010B500F001F810BDC6
:104360000CB50020019000903348006840F4803084
:104370003149086000BF3048006800F40030009008
:104380000198401C0190009818B90198B0F5A06FF1
:10439000F1D12948006800F4003010B101200090EC
:1043A00001E0002000900098012843D123480068D4
:1043B00040F01000214908600846006820F0030022
:1043C00008600846006840F0020008601A4840682B
:1043D000194948600846406848600846406840F40B
:1043E000806048600846406820F47C1048600846B9
:1043F000406840F4A81048600846006840F08070AB
:10440000086000BF0C48006800F000700028F9D078
:104410000948406820F003000749486008464068A2
:1044200040F00200486000BF0348406800F00C0004
:104430000828F9D10CBD0000001002400020024005
:1044400070B505460C46FFF7D7F825B1012D13D0FE
:10445000022D3BD129E01F4890F8D00000B136E092
:1044600001201C4981F8D0001B4908604FF47A7183
:104470000920FDF7DDFB2AE0164890F8D00000B1D6
:1044800025E00120134981F8D00013490860022C6F
:1044900005D14FF47A710B20FDF7CAFB04E04FF40D
:1044A0007A710A20FDF7C4FB11E00A4890F8D000A9
:1044B00000B10CE00120074981F8D00006490860EE
:1044C0004FF47A710820FDF7B3FB00E000BF00BF96
:1044D00070BD0000EC0A0020380000202DE9F041FA
:1044E00005460E469046144C00271CE02068B8B9DB
:1044F00025B1012D03D0022D03D101E000BF00BF83
:1045000004E000202060401EBDE8F08100BFE660AE
:104510002661C4F8148065600120206078B2F3E75A
:10452000781CC7B22834052FE0DB04A0FFF7A0F801
:104530004FF0FF30E8E70000E00D0020B6A8CAB158
:10454000C6F7D7CAD4B4B2BBD7E32CC9EAC7EBB21B
:10455000BBB3C9B9A60000002DE9F04104460E46E0
:10456000174698464FF0FF35C4B12068401C28B16B
:1045700012A0FFF77DF82846BDE8F081F0B2424670
:104580003946FFF7ABFF05462560002D13DB05EB31
:104590008500124901EBC00084600CE0F0B2424695
:1045A0003946FFF79BFF0546002005EB85010B4AC6
:1045B00002EBC10188602846DEE70000B6A8CAB158
:1045C000C6F7B2BBCEAA2D312CCDA3D6B9BAF3D63D
:1045D000D8D0C2C6F4D3C30A00000000E00D00200A
:1045E0002DE9FF5F0746884691460E9D4A464146A3
:1045F0003846039BFFF7B0FF0446002C25DB284616
:10460000FBF7B0FE82464FF00F0BDA4501DD58464E
:1046100000E05046064604EB84010E4A02EBC1015D
:1046200001F1180032462946FBF7BBFE002104EBDE
:104630008400084A02EBC0001830815523464A46E0
:1046400029460548FFF714F800BF204604B0BDE82E
:10465000F09F0000E00D0020D06A0008002027E055
:10466000002100EB8002144B43F8321000EB800174
:104670001A4602EBC101896839B14FF0FF3100EBF6
:10468000800203EBC20292681160002100EB8002FD
:10469000094B03EBC202916000EB80011A4602EB6A
:1046A000C10100228A61CA610A624A62411CC8B221
:1046B0000528D5DB70470000E00D002008B5134841
:1046C000006820F04000114908600020104908608F
:1046D0000E48006840F020000C4908600846008839
:1046E0000C49088000BF0CA00C4BBF220CA100900D
:1046F0000FA0FEF7BDFF19A01C4B47F2305201215D
:1047000000900020FFF76CFF00BF08BD4C000020A8
:10471000A88121422C000020300000009969000887
:104720004170705C4945445F4354524C2E43000035
:1047300046696C6520257320204C696E65202564D0
:1047400020257320537461727454696D65725769C2
:1047500074684E616D652825732900004A75646789
:10476000654469616E48756F0000000039360008C5
:1047700010B500200D4908600D48006820F00200C7
:104780000B4908600846006840F0010008600846D0
:10479000008808490880084890F8CD0020F0020001
:1047A000054981F8CD00FDF7C3FF10BD808121428E
:1047B0004C0000202C000020EC0A002000200A49B8
:1047C00008600A48006820F01000084908600846A0
:1047D000008807490880074890F8CD0020F00800BD
:1047E000044981F8CD007047888121424C000020A7
:1047F0002C000020EC0A002008B5002012490860B7
:104800001248006820F00800104908600846008837
:104810000F4908800F4890F8CD0020F001000D49A5
:1048200081F8CD000C480068401C60B100BF0BA0AF
:104830000D4B6A220DA1009010A0FEF719FF06484B
:1048400001F058FE00BF08BD848121424C000020C9
:104850002C000020EC0A0020480000202654696D3E
:1048600065724A53000000007E6900084170705C68
:104870004945445F4354524C2E43000046696C65E1
:1048800020257320204C696E652025642025732027
:1048900053746F7054696D65722825732900000088
:1048A00008B500200949086009480068401C60B14B
:1048B00000BF08A00B4B4B220BA100900EA0FEF7EF
:1048C000D7FE034801F016FE00BF08BD9401224246
:1048D000440000202654696D657253746F70574A06
:1048E000420000006B6900084170705C4945445FFC
:1048F0004354524C2E43000046696C6520257320BA
:10490000204C696E652025642025732053746F70D8
:1049100054696D65722825732900000010B50146A1
:1049200000200FE000EB4002084B03EBC2021269CB
:104930008A4206D1002200EB4003044C44F83320A5
:1049400002E0401C0C28EDD300BF10BDAC000020DD
:1049500008480068012804D107480068401C06493F
:10496000086001200349086004480068401C0349AE
:1049700008607047CC010020D0010020D401002045
:1049800010B51348006840F001001149086008465E
:104990004068104908400E494860084600680E49C2
:1049A00008400B4908600846006820F48020086031
:1049B0000846406820F4FE0048604FF41F008860FD
:1049C000FFF7CAFC4FF000600449086010BD00000A
:1049D000001002400000FFF8FFFFF6FE08ED00E0C7
:1049E00008B53B480068002846DD39480068401E8D
:1049F0003749086000283FD13649086036480068CA
:104A0000401C354908600846007800F00100086045
:104A1000FEF7A0FC3149304A126841F822000968CB
:104A20002E4A5268881A002801DB014600E0414204
:104A30002B4A116000BF2BA02E4B40F2D9322EA181
:104A4000009031A0FEF714FE384801F053FD00BF7E
:104A500000BF24A0274B40F2DA3227A1009034A0F7
:104A6000FEF706FE3DA0404B41F288320121009046
:104A70002E48FFF7B5FD00BF3C480068002813DD55
:104A800000BF3BA01B4B4FF478721BA1009028A0E5
:104A9000FEF7EEFD31A0344B41F288320121009047
:104AA0003748FFF79DFD11E035480068401C68B1AC
:104AB00000BF2FA00F4B40F2E6320FA1009012A0D2
:104AC000FEF7D6FD2E4801F015FD00BF08BD000021
:104AD00010000020900121421C0000201400002042
:104AE00020000020265265496E697454696D657214
:104AF00000000000646900084170705C414453315B
:104B00003236322E4300000046696C652025732042
:104B1000204C696E652025642025732053746F70C6
:104B200054696D6572282573290000002400002057
:104B300046696C6520257320204C696E65202564CC
:104B400020257320537461727454696D65725769BE
:104B500074684E616D65282573290000496E69747B
:104B60004144533132363200653300080C000020D6
:104B7000265265496E697454696D65723200000091
:104B80002800002000B50F48007818B101200E4918
:104B900008600DE000200C4908600C480068401EC9
:104BA0000A4908600846006810B90220FFF7B6FEFF
:104BB0000448007808B9012000E00020014908708D
:104BC00000BD0000D8010020AC812142DC010020A2
:104BD0000B480078401CC0B2094908700A2190FBBC
:104BE000F1F201FB1200064908700846007800281F
:104BF00001DD012000E0002002490860704700004C
:104C0000E0010020B401224210B53548007800B917
:104C100010BD344C002032490870334908702078A8
:104C200032490978884202D02078FF2853D1A178F0
:104C3000091DC8B22146FEF70BFD00284BD1207894
:104C4000FF2805D16078022845D1FDF793FB42E0AB
:104C50006078092800D000BF6078132839D2DFE8D7
:104C600000F0380A0D1011121314171A20232629E8
:104C70002F32351D2C00FDF74BFB2BE0FDF77AFBA7
:104C800028E027E026E025E024E0FDF719FB21E0FD
:104C9000FDF774F91EE0FDF7B3FA1BE0FDF7D2F95A
:104CA00018E0FDF7B5F815E0FDF756F812E0FDF74E
:104CB00029F80FE0FDF77AF80CE0FDF78BFB09E02F
:104CC000FDF7FCF806E0FDF72DF903E0FDF7CAF863
:104CD00000E000BF00BF00200549087000BF97E753
:104CE00058000020D40C002056000020EC0A0020C0
:104CF0005700002010B51F48006850B11D480068DB
:104D0000401E1C4908600846006810B901201A4975
:104D100008601A48006878B1194801680068401EA8
:104D2000174A106041B9002014490860012240F27E
:104D30002771144801F0FAF81348006858B1134875
:104D400001680068401E114A106021B9FEF7CEFBD1
:104D500000200D4908600E48006848B10D48016800
:104D60000068401E0B4A106011B900200849086015
:104D700010BD00005C0000205800002060000020F2
:104D80006400002000380140680000206C00002012
:104D9000700000207400002010B5FEF7BDFA44B288
:104DA000124890F8CC0040F08000104981F8CC0007
:104DB000082000F0E5FE58B9092000F0E1FE38B9FE
:104DC0000A2000F0DDFE18B90B2000F0D9FE08B172
:104DD000012000E0002040B93CB1044890F8CC002C
:104DE00040F00100014981F8CC0010BDEC0A002020
:104DF00038B5B84800680A2878D2DFE800F07705AF
:104E00002077789AD1FDFCFBB34890F8CD0000F0F4
:104E1000020098B9FCF750FFAF4890F8CD0040F081
:104E20008000AD4981F8CD000120FCF72BFFFDF794
:104E300007FCFDF7DFFB0220A649086047E1A64812
:104E400090F8CD0000F0010000284ED100BFA3A0D3
:104E5000A34B4FF4C272A3A10090A6A0FEF708FCDA
:104E6000AFA0B14B4EF66022012100900020FFF769
:104E7000B7FB00BF984890F82C0001281AD10420F5
:104E80009449086000BF95A0954B4FF4C57295A159
:104E9000009098A0FEF7ECFBA4A000908E48007F45
:104EA0004EF6602100FB01F2A24B01210020FFF72A
:104EB00097FB1AE005208749086000BF87A0884B50
:104EC0004FF4C87287A100908AA0FEF7D1FB9AA088
:104ED00000908148407F4EF6602100FB01F2984B24
:104EE00001210020FFF77CFB00BFF0E0EEE07A48F4
:104EF00090F8CE0000F00200D0B10520754908609E
:104F000000BF76A0764B4FF4CD7276A1009079A0C9
:104F1000FEF7AEFB88A000906F48407F4EF6602100
:104F200000FB01F2864B01210020FFF759FB00BF77
:104F3000CDE0694890F8CE0000F0040000282ED0A3
:104F40000620644908600220FCF79CFEFDF774FA15
:104F500000BF62A0624B4FF4D27262A1009065A0C4
:104F6000FEF786FB77A07A4B7A4A01210090002059
:104F7000FFF736FB00BF00BF77A0594B4FF4D37249
:104F800058A100905BA0FEF773FB77A0784B4EF61C
:104F90006022012100907748FFF722FB00BF96E0D6
:104FA0004D4890F8CD0000F0040030BB4A48406BFB
:104FB0004949096C441A4848456AAC420ADB90F8F2
:104FC000CD0040F01000444981F8CD000720414950
:104FD000086020E0404890F8CD0040F020003E49B5
:104FE00081F8CD00084690F8CD0020F0800081F8CF
:104FF000CD0003E056E03FE00EE00CE0FFF72EFBB3
:10500000FFF7FAFBFFF75AFBFFF7D8FBFDF780FA33
:105010000920304908605AE02F4890F8CE0000F08F
:105020002000002827D008202A4908602A4890F844
:105030002C00012817D100BF28A0294B40F2C7122D
:1050400028A100902BA0FEF713FB4BA00090224854
:10505000807F4EF6602100FB01F2494B01210020C8
:10506000FFF7BEFA07E01C4890F8CE0040F0400081
:10507000194981F8CE002AE0174890F8CE0000F0D8
:10508000400070B1092013490860134890F8CD0022
:1050900020F08000104981F8CD00FFF78FFBFDF76D
:1050A00037FA14E00C4890F8CD0000F0020060B927
:1050B0000020084908600320FCF7E4FD0920FFF701
:1050C0002DFC0020044981F8D00000E000BF00BFA3
:1050D00038BD000038000020EC0A0020300000003D
:1050E000B16900084170705C4945445F4354524CBB
:1050F0002E43000046696C6520257320204C696EA4
:105100006520256420257320537461727454696D81
:105110006572576974684E616D65282573290000B2
:1051200052656164746A00007D3B000852656164E9
:1051300054300000353A0008526561647430000054
:10514000613B000852656164543134300000000056
:10515000513A0008A08601002667635265616454D5
:105160006954696D6572000052656164546900009C
:105170006D3A00083000002052656164546E0000F2
:10518000453B000810B51B480068C4B2B4B11A48CA
:105190000078844205D01848047000201749086040
:1051A00026E016480068042802D904201349086044
:1051B00012480068401C1149086019E00F48006857
:1051C000042815D900200D4908600B4800780C49C7
:1051D0000C4A127888540B480078401C0A2190FB36
:1051E000F1F201FB1200074908700120FCF74AFDAB
:1051F00010BD000030012242780000207C00002019
:10520000D40D00208000002038B5A74800680B2886
:1052100077D2DFE800F0F70621767799BDF8F5F44C
:105220004400A24890F8CD0000F0020098B9FCF7C5
:1052300043FD9E4890F8CD0040F080009B4981F8E6
:10524000CD000120FCF71EFDFDF7FAF9FDF7D2F9BC
:1052500002209549086024E1944890F8CD0000F0C0
:10526000010000281AD10A208F49086000BF90A0D1
:10527000904B40F2592290A1009093A0FEF7F8F9CC
:105280009CA000908948007F4EF6602100FB01F24F
:105290009A4B01210020FFF7A3F900BF01E18348E9
:1052A00090F8CE0000F00100002829D0FFF786FA20
:1052B0007E4890F8CC0000F0800020B97B4890F840
:1052C0002D0000281CD0FDF795F900BF78A0794B80
:1052D0004FF4197278A100907BA0FEF7C9F988A05D
:1052E00000907248007F4EF6602100FB01F2864B71
:1052F00001210020FFF774F900BF04206A4908600B
:10530000CFE0CDE0694890F8CE0000F00200D0B1C7
:1053100005206549086000BF65A0664B40F26E221B
:1053200065A1009068A0FEF7A3F978A000905F48FF
:10533000407F4EF6602100FB01F2764B01210020F8
:10534000FFF74EF900BFACE0584890F8CE0000F0EF
:10535000040000281BD00620534908600220FCF7F7
:1053600091FCFDF769F800BF6BA0524B4FF41E7221
:1053700051A1009054A0FEF77BF96BA06C4B4EF648
:105380006022022100906B48FFF72AF900BF88E0F5
:10539000464890F8CD0000F0040078BB4348406BCD
:1053A0004249096C441A4148456AAC420ADB90F80C
:1053B000CD0040F010003D4981F8CD0007203A496A
:1053C00008601BE0394890F8CD0040F020003749D4
:1053D00081F8CD00084690F8CD0020F0800081F8DB
:1053E000CD00FFF73BF9FFF707FAFFF767F9FFF783
:1053F000E5F9FDF78DF809202B49086051E03AE006
:1054000023E000E04BE0294890F8CE0000F02000B7
:10541000D0B108202449086000BF25A0254B40F2E8
:10542000972225A1009028A0FEF722F942A0009023
:105430001E48807F4EF6602100FB01F2404B0121A7
:105440000020FFF7CDF800BF2BE0184890F8CE0001
:1054500000F0400070B1092013490860134890F82B
:10546000CD0020F08000114981F8CD00FFF7A6F9AA
:10547000FDF74EF815E00D4890F8CD0000F0020061
:1054800060B90020084908600320FCF7FBFB0020FE
:10549000064981F8D0000B20FFF740FA01E000E058
:1054A00000BF00BF38BD000038000020EC0A00201B
:1054B00030000000CC6900084170705C4945445FD1
:1054C0004354524C2E43000046696C6520257320DE
:1054D000204C696E65202564202573205374617209
:1054E0007454696D6572576974684E616D652825DD
:1054F0007329000052656164746A00007D3B0008F6
:105500005265616454300000353A000852656164A8
:1055100074300000613B0008266763526561645483
:105520006954696D657200005265616454690000D8
:105530006D3A00083000002052656164546E00002E
:10554000453B000838B57F4800680A287CD2DFE870
:1055500000F0F50520F5F55794F5CBE17A4890F881
:10556000CD0000F0020098B9FCF7A6FB764890F851
:10557000CD0040F08000744981F8CD000120FCF797
:1055800081FBFDF75DF8FDF735F802206D490860F5
:10559000D5E06D4890F8CD0000F0010000282ED134
:1055A00005206849086000BF68A0694B40F2FF12FF
:1055B00068A100906BA0FEF75BF875A0764B4EF6E5
:1055C0006022012100900020FFF70AF800BF00BF11
:1055D0005EA05F4B4FF400725EA1009061A0FEF7E9
:1055E00047F86EA000905848007F4EF6602100FBFF
:1055F00001F26C4B01210020FEF7F2FF00BF9EE09C
:10560000514890F8CE0000F00400002834D0062065
:105610004C4908600220FCF735FBFCF70DFF00BF8A
:1056200061A04B4B40F20A224AA100904DA0FEF728
:105630001FF861A0634B644A022100906348FEF7A3
:10564000CFFF00BF00BF00E078E061A0404B4FF407
:10565000037240A1009043A0FEF70AF860A00090FA
:105660003948007F4EF6602100FB01F25E4B0121BC
:105670005E48FEF7B5FF00BF61E0334890F8CD000B
:1056800000F0040078BB3048406B2F49096C441A85
:105690002D48456AAC420ADB90F8CD0040F010007E
:1056A000294981F8CD000820264908601BE02648DA
:1056B00090F8CD0040F02000234981F8CD00084645
:1056C00090F8CD0020F0800081F8CD00FEF7C6FFF5
:1056D000FFF792F8FEF7F2FFFFF770F8FCF718FFFC
:1056E0000920184908602AE0174890F8CE0000F019
:1056F000200070B1092013490860134890F8CD00CC
:1057000020F08000104981F8CD00FFF757F8FCF732
:10571000FFFE14E00C4890F8CD0000F0020060B9E4
:105720000020084908600320FCF7ACFA0A20FFF7C4
:10573000F5F80020044981F8D00000E000BF00BF68
:1057400038BD000038000020EC0A002030000000C6
:10575000BF6900084170705C4945445F4354524C36
:105760002E43000046696C6520257320204C696E2D
:105770006520256420257320537461727454696D0B
:105780006572576974684E616D652825732900003C
:1057900052656164746A00007D3B00085265616473
:1057A00074300000613B00082667635265616454F1
:1057B0006954696D6572000052656164543134301A
:1057C00000000000513A0008A086010030000020CF
:1057D00026676352656164746E54696D657200007A
:1057E00052656164746E0000993B0008340000202B
:1057F00010B52C48006810B900F051FF50E02A485D
:105800000068A0B1002410E004EB4400274901EB3C
:10581000C000806824490968401A04EB4401234A07
:1058200002EBC1018860601CC4B20C2CECD30020D8
:105830001C4908601C49086000242FE004EB440068
:105840001A4951F8300000B926E004EB440017492A
:1058500001EBC0008068401E04EB4401134A02EBD8
:10586000C1018860002816DC04EB4400114601EBFE
:10587000C000806804EB440102EBC101C968084420
:1058800004EB440102EBC101886004EB440102EB2C
:10589000C1014869804700BF601CC4B20C2CCDD345
:1058A00010BD0000CC010020D0010020AC00002081
:1058B00038B58F4800680A287ED2DFE800F07D0501
:1058C000207D4B6D93CAECFC8A4890F8CD0000F027
:1058D000020098B9FCF7F0F9864890F8CD0040F046
:1058E0008000844981F8CD000120FCF7CBF9FCF75A
:1058F000A7FEFCF77FFE02207D490860F5E07D48A9
:1059000090F8CC0020F001007A4981F8CC000846DC
:1059100090F8CD0000F0010000281AD1042074494D
:10592000086000BF74A0754B40F2D12274A10090B2
:1059300077A0FDF79DFE81A000906E48007F4EF697
:10594000602100FB01F27F4B01210020FEF748FEA1
:1059500000BFCAE0674890F8CE0000F00200D0B166
:1059600005206349086000BF63A0644B40F2DA225F
:1059700063A1009066A0FDF77BFE73A000905D48D8
:10598000407F4EF6602100FB01F2714B01210020A7
:10599000FEF726FE00BFA8E0564890F8CE0000F0C3
:1059A000040000281DD00620514908600220FCF7A1
:1059B00069F9FCF741FD00E096E000BF65A04F4BA0
:1059C0004FF439724EA1009051A0FDF751FE65A031
:1059D000664B4EF66022022100906548FEF700FEFD
:1059E00000BF82E0434890F8CD0000F0040078BB8F
:1059F0004048406B3F49096C441A3E48456AAC42F6
:105A00000ADB90F8CD0040F010003A4981F8CD0053
:105A10000720374908601BE0364890F8CD0040F079
:105A20002000344981F8CD00084690F8CD0020F0E0
:105A3000800081F8CD00FEF711FEFEF7DDFEFEF7D7
:105A40003DFEFEF7BBFEFCF763FD09202849086018
:105A50004BE0284890F8CE0000F02000D0B108209C
:105A60002349086000BF24A0244B40F2023224A145
:105A7000009027A0FDF7FCFD3EA000901D48807F10
:105A80004EF6602100FB01F23C4B01210020FEF7A5
:105A9000A7FD00BF29E0174890F8CE0000F04000B5
:105AA00080B1092012490860124890F8CD0020F01A
:105AB0008000104900E006E081F8CD00FEF77EFE90
:105AC000FCF726FD11E00B4890F8CD0000F0020035
:105AD00048B90320FCF7D6F80820FEF71FFF002086
:105AE000044981F8D00000E000BF00BF38BD0000CD
:105AF00038000020EC0A002030000000D9690008BE
:105B00004170705C4945445F4354524C2E43000041
:105B100046696C6520257320204C696E65202564DC
:105B200020257320537461727454696D65725769CE
:105B300074684E616D6528257329000052656164A3
:105B400054300000353A000852656164743000003A
:105B5000613B000826676352656164546954696D4E
:105B60006572000052656164546900006D3A000876
:105B70003000002052656164546E0000453B00080F
:105B8000024600210DE001EB4100084B03EBC00091
:105B90000069904204D101EB410053F83000704796
:105BA000491C0C29EFD30020F9E70000AC000020CD
:105BB00070B5234C002540E0206800B93AE0206928
:105BC000401E2061002834DC606820B101280CD020
:105BD000022815D102E00020206014E0D4E903106F
:105BE00008442061606980470DE000202060A068C3
:105BF00018B14FF0FF30A16808606069804702E08B
:105C00000020206000BF00BF05EB85000C4901EBC0
:105C1000C00000F1180229460AA0FDF729FD6068BE
:105C2000022806D0002005EB8501054A02EBC101E0
:105C3000087600BF681CC5B22834052DBCDB70BDDA
:105C4000E00D0020B6A8CAB1C6F725642C2573BAAA
:105C5000AFCAFDB3C9B9A6D6B4D0D00A00000000BF
:105C600010B540F22551284800F0BAF878B1142058
:105C7000264908602448001D0088C1B224480278E3
:105C80000078401C224B18702248815400BF40F21B
:105C900027711D4800F0A4F8E8B11F4800781F499B
:105CA000097888420BDA1C4801780078401C1A4AAF
:105CB00010701B48405C1449091D08800BE000224D
:105CC00040F22771104800F031F9012240F22661BC
:105CD0000D4800F02BF940F226610B4800F080F8E7
:105CE00088B1002240F22661074800F01FF9002029
:105CF0000C49086001200C49086002200B4908602B
:105D000000200B49086010BD003801405C000020F5
:105D100056000020D40C0020540000205500002024
:105D2000D40B0020A001214270000020740000204C
:105D30006800002070B504460D46154884420BD01B
:105D40001448844208D01448844205D01348844241
:105D500002D01348844200D104E04FF4B17111A085
:105D600000F09AFC0DB1012D00D104E040F2631166
:105D70000CA000F091FC25B1A08940F40050A08156
:105D800004E0A0894DF6FF710840A08170BD0000BD
:105D9000003801400044004000480040004C0040F2
:105DA000005000404C69627261726965735C5354C3
:105DB0004D3332463130785F537464506572697088
:105DC000685F4472697665725C7372635C73746D4C
:105DD0003332663130785F75736172742E63000000
:105DE0002DE9F04705460C4600270026B046B1468F
:105DF0003A4885420BD03A48854208D03948854216
:105E000005D03948854202D03848854200D104E0A7
:105E100040F2C13136A000F03FFC282C20D040F2E7
:105E2000277084421CD040F22660844218D040F291
:105E30002550844214D040F22440844210D040F6D1
:105E4000460084420CD040F66A10844208D0B4F573
:105E5000587F05D0B4F5187F02D0B4F5B07F00D1DB
:105E600004E040F2C23122A000F016FC40F66A10B5
:105E700084420ED11948854205D01948854202D086
:105E80001848854200D104E040F2C63118A000F065
:105E900003FCC4F3421804F01F06012000FA06F6C2
:105EA000B8F1010F02D1A889064007E0B8F1020F4E
:105EB00002D1288A064001E0A88A06402712012064
:105EC00000FA07F7288807401EB117B14FF0010903
:105ED00001E04FF000094846BDE8F0870038014076
:105EE0000044004000480040004C0040005000408A
:105EF0004C69627261726965735C53544D3332460A
:105F00003130785F5374645065726970685F4472B1
:105F1000697665725C7372635C73746D333266317B
:105F200030785F75736172742E6300002DE9F0475D
:105F300005460C4617464FF00008C246C1460026EB
:105F4000384885420BD03848854208D037488542CA
:105F500005D03748854202D03648854200D104E05A
:105F600040F2891134A000F097FB282C19D040F2A0
:105F70002770844215D040F22660844211D040F24E
:105F8000255084420DD040F22440844209D040F68E
:105F90004600844205D040F66A10844201D0602C4D
:105FA00000D104E04FF4C57123A000F075FB0FB1E0
:105FB000012F00D104E040F28B111FA000F06CFB18
:105FC00040F66A1084420ED11648854205D0164824
:105FD000854202D01548854200D104E040F28F117D
:105FE00015A000F059FB2E46C4F3421804F01F0A16
:105FF000012000FA0AF9B8F1010F01D10C3605E0D1
:10600000B8F1020F01D1103600E0143627B1306824
:1060100040EA0900306003E0306820EA090030609F
:10602000BDE8F087003801400044004000480040CF
:10603000004C0040005000404C696272617269651A
:10604000735C53544D3332463130785F537464502F
:1060500065726970685F4472697665725C737263B9
:106060005C73746D3332663130785F75736172744E
:106070002E6300002DE9F04786B005460C46002649
:10608000B24600BFB14600276B4885420BD06B4833
:10609000854208D06A48854205D06A48854202D0C8
:1060A0006948854200D103E0B82168A000F0F4FA05
:1060B000206820B174492068884200D203E0B921E9
:1060C00062A000F0E9FAA08818B1A088B0F5805F5E
:1060D00000D103E0BA215DA000F0DEFAE08858B1FB
:1060E000E088B0F5805F07D0E088B0F5005F03D0AE
:1060F000E088B0F5405F00D103E0BB2153A000F081
:10610000CBFA208938B12089B0F5806F03D020897F
:10611000B0F5C06F00D103E0BC214CA000F0BCFA88
:1061200060894FF6F371084010B9608900B103E04F
:10613000BD2146A000F0B0FAA08958B1A089B0F501
:10614000807F07D0A089B0F5007F03D0A089B0F58B
:10615000407F00D103E0BE213CA000F09DFAA08961
:1061600068B13548854205D03448854202D034486C
:10617000854200D103E0C22134A000F08DFA2F4601
:106180002E8A4CF6FF700640E08806432E82AE89C8
:106190004EF6F3100640A088218908436189084320
:1061A0000643AE81AE8A4FF6FF400640A089064303
:1061B000AE8201A8FDF762FB1F48874202D1DDF8DD
:1061C00010A001E0DDF80CA0A88900F4004040B167
:1061D0000AEBCA0000EB0A1021684900B0FBF1F895
:1061E00007E00AEBCA0000EB0A1021688900B0FB47
:1061F000F1F86420B8FBF0F006013009642101FBDE
:106200001089A88900F4004040B1322000EBC90099
:10621000B0FBF1F000F00700064308E0322000EB8D
:1062200009106421B0FBF1F000F00F0006432E814D
:1062300006B0BDE8F087000000380140004400408F
:1062400000480040004C0040005000404C69627221
:1062500061726965735C53544D3332463130785FF7
:106260005374645065726970685F447269766572D0
:106270005C7372635C73746D3332663130785F7552
:10628000736172742E63000021AA440000BFFEE710
:1062900010B5124C02202061606111A0A061134969
:1062A000E1614FF4806121620021A1626162E162DB
:1062B0000BA0A0640E49E164102121650021A165B5
:1062C0006165E1650BA1E01DFAF728F80AA12046F7
:1062D000FAF724F82020A07110BD0000B8120020A9
:1062E0005465726D696E616C00000000A80E00209C
:1062F000A81200205254540053454747455200000D
:1063000010B501460A69CB689A4204D88C68641EAD
:10631000E41AA01801E0D41A601E10BD2DE9FC5F3C
:1063200006460F4692469846DDE90C45002F01DAF5
:10633000784200E0384683464FF0010903E09BFBBA
:10634000FAFB09F10109D345F9DAC84500D9C1467C
:1063500034B1002F03DB05F00400042800D1641ED3
:1063600005F0020010B1B8F1000F11D005F00100E6
:1063700070B96CB108E0641E2021304600F0F0F8DE
:10638000F068002800DA02E00CB1A145F3D300BFA9
:10639000F068002836DB002F05DA7F422D213046D9
:1063A00000F0DEF807E005F00400042803D12B21FB
:1063B000304600F0D5F8F068002823DB05F0020035
:1063C000022814D105F0010088B9B8F1000F0ED1F0
:1063D0006CB108E0641E3021304600F0C1F8F0686E
:1063E000002800DA02E00CB1A145F3D300BFF06849
:1063F000002807DB4346524639463046CDE9004582
:1064000000F002F8BDE8FC9F2DE9FC5F804689465C
:1064100015461E460C9CCDF804900127BB4605E0AE
:106420000198B0FBF5F001900BF1010B0198A84227
:10643000F6D25E4500D9B3460D9800F00100D0B900
:10644000CCB10D9800F00200022803D116B930201B
:10645000009001E02020009009E0641E4046009971
:1064600000F07EF8D8F80C00002800DA02E00CB149
:10647000A345F2D300BFD8F80C00002835DB09E0B3
:10648000012E01D9761E04E0B9FBF7FAAA4500D225
:1064900001E06F43F4E700BF00BFB9FBF7FA0AFB66
:1064A0001799134810F90A10404600F059F8D8F827
:1064B0000C00002800DA03E0B7FBF5F7002FECD161
:1064C00000BF0D9800F0010078B174B109E0641EBE
:1064D0002021404600F044F8D8F80C00002800DAEB
:1064E00002E00CB1A345F2D300BFBDE8FC9F000061
:1064F000E769000810B504462068052802DA20681C
:10650000401C10B94FF0FF3010BD206800EB800038
:10651000094B03EBC00000F1180208A02168FDF749
:10652000A7F80020216801EB8101034A42F83100FD
:10653000401E20600020E7E7E00D0020B6A8CAB1A9
:10654000C6F72564CDA3D6B9B3C9B9A62C25732047
:1065500020B2BBD4D9B1BBD6B4D0D00A0000000061
:1065600070B504460E46A568681C6168814206D372
:1065700020684655681CA060E068401CE060D4E9D3
:10658000011088420DD1A26821682069FDF730FB17
:10659000A168884203D04FF0FF30E06001E00020A6
:1065A000A06070BD2DE9F0470446894617464FF0BC
:1065B000000AE56800BFD4F81080A84503D9A8EB0D
:1065C0000500461E04E0A5EB0800401CA1680E1A59
:1065D000A068401BB04201D9304601E0A068401BD2
:1065E0000646BE4201D2304600E0384606466168A3
:1065F000481932464946F9F7D4FEB244B144BF1BAC
:106600003544A068A84200D10025E560002FD2D112
:106610005046BDE8F0872DE9F04704468946154607
:10662000E668A068871BAF4208D9616888192A46C6
:106630004946F9F7B6FE7019E06010E0B8466168A7
:10664000881942464946F9F7ACFEA5EB070809EB65
:10665000070142466068F9F7A4FEC4F80C80BDE863
:10666000F087490050EAC12018BF04204A0D18BF26
:1066700040F0010040F2FF72B2EB515F08BF40F002
:106680000200012808BF0520704730380A2801D2CF
:10669000012070470020704700BF00BFFEE7704731
:1066A00008B528208DF803004FF48050ADF80000A5
:1066B00003208DF8020069460148FCF7D3FB08BDB2
:1066C0000010014072B61048FDF7D8F800F082F8CB
:1066D000FDF770FAFCF758FEFCF7AAFEFCF76AFE1D
:1066E000FCF704FF6420FCF775F8FCF73BFE012083
:1066F000FBF7C8FAFDF7B2FFFCF79CFF62B601E0BA
:10670000FFF776F8FCE70000C00B00202448806902
:1067100040F0040022498861224823490860234848
:10672000091D08601E48806940F008001C49886106
:106730001F48204908602048091D086018488069E2
:1067400040F01000164988614FF40C101B49086096
:106750001B4848601248806940F020001049886159
:106760001848194908600020091D08600C48806914
:1067700040F040000A4988614FF0443013490860F6
:10678000091D08600648806940F08000044988615E
:106790004FF088300E490860091D086070470000FE
:1067A000001002404444233400080140B1444344F3
:1067B00022224244000C01404422B44B001001400C
:1067C0000800680611121111001401400018014060
:1067D000001C014010B500BF1F48204948602048F8
:1067E000086000BF00BF1D48006800F002000028DC
:1067F000F9D000BF1948006800F400300028F9D033
:1068000000BF1648006800F000700028F9D000BFF3
:106810001248406800F00C000828F9D100BF00BF02
:1068200000201049086000BF00BF41F657304FF00C
:10683000E021486102200861002088610846006963
:1068400040F00100086100BF00BF00BFFFF75EFF1E
:1068500000F00AF810BD00000228150000100240E8
:106860008300090108ED00E02348806940F0010041
:10687000214988612148406820F004001F49486090
:106880001D48806940F004001B4988611C4800686D
:1068900020F47F601A4908600846006840F0B000A4
:1068A00008600846006840F480600860124880690B
:1068B00040F480401049886140F2B250114908808C
:1068C0000020091D0880091D0880081F0088091F75
:1068D000088000200B490C3108800A48001D008800
:1068E00040F00C000749091D08800846008840F464
:1068F0000050088070470000001002400000014076
:10690000040801400838014010B500290AD0087871
:10691000002807D005487844FAF780FC002801D009
:10692000002010BD0248784410BD00001E02000087
:106930001602000010B500290AD00878002807D0F8
:1069400005487844FAF76AFC002801D0002010BD01
:106950000248784410BD00000E020000060200004C
:10696000FAF7E9B95461736B41490053746F705879
:10697000484200436F6E74726F6C58484200537403
:106980006F704A5300436F6E74726F6C4A530043CA
:106990006F6E74726F6C46530053746F704448008E
:1069A000436F6E74726F6C44480052656164546941
:1069B000005461736B47756F4269616F51450054B4
:1069C00061736B4B75616953755145005461736B0D
:1069D0004B7561695375414B005461736B52756916
:1069E00046616E67514500303132333435363738C1
:1069F00039414243444546000000000000000000C9
:106A000030313233343536373839414243444546E4
:106A100040305800303132333435363738396162DE
:106A200063646566403078000400000800000000E0
:106A30000000000200010000100000000240000001
:106A4000000000A00000000005400000000000C899
:106A5000000000000C4000000000409C000000000E
:106A6000194000000020BCBE0000000034400000BF
:106A7000BFC91B8E00000004B5400000504BCFD0B2
:106A80006607E2CF010000006C4100003E8251AA7F
:106A9000DFEEA73401000000D9420000DCB5A0E21F
:106AA0003A301F97FFFFFFFFB4450000FD25A0C847
:106AB000E9A3C14FFFFFFFFFFF3F00000000008080
:106AC00000000000FF3F0000000000800000000008
:106AD0000A2063616C6C2025732046756E637469AF
:106AE0006F6E2077696C6C206578656375746520BE
:106AF000206166746572202564206D73206C61745A
:106B00006572202C54696D65726964203D2025648E
:106B10000A000000606C000800000020E401000092
:106B20006C010008EC6C0008E4010020E417000090
:106B3000C80100081C00000043000000F8FFFFFF30
:106B40000C0000000E0000000F0000002E000000EE
:106B50001001000043000000F8FFFFFF004040402C
:106B60004040404040404141414141404040404020
:106B700040404040404040404040404040050202CC
:106B8000020202020202020202020202022020208B
:106B900020202020202020020202020202029090E7
:106BA00090909090101010101010101010101010E5
:106BB0001010101010101010020202020202888839
:106BC0008888888808080808080808080808080845
:106BD000080808080808080802020202400000002D
:106BE00000000000000000000000000000000000A5
:106BF0000000000000000000000000000000000095
:106C00000000000000000000000000000000000084
:106C10000000000000000000000000000000000074
:106C20000000000000000000000000000000000064
:106C30000000000000000000000000000000000054
:106C40000000000000000000000000000000000044
:106C50000000000000000000000000000000000034
:106C600001100213015AFF01E90C091620012E1927
:106C70002F7C7E5603806808020304060708090C6F
:106C800069102D020406089CE90413B15B6A08B878
:106C90001AE8462904320213854B79305A640429D4
:106CA000659AD11869383205CBF54C183214320682
:106CB000DA09181A90093204CBE1491832C8320DAA
:106CC0000B10994D482A0C908A51A8412990320AFC
:106CD0000B104555182A0B780A10521832091AF170
:0C6CE00060E91829114BB158180114008C
:0400000508000131BD
:00000001FF
